:020000040800F2
:1000000000070020F1010008CD2D0008852D000813
:10001000AD2D0008852D0008A52D0008F30100086E
:10002000F3010008F3010008F3010008693E00082D
:10003000F3010008F3010008F3010008F3010008D0
:10004000F3010008F3010008F3010008F3010008C0
:10005000F3010008F3010008F963000821640008B7
:10006000496400087164000899640008F3010008FD
:10007000F3010008F3010008F3010008F301000890
:10008000F3010008F3010008F3010008152D000832
:10009000252D0008392D0008F3010008C16400086F
:1000A000F3010008F3010008F3010008F301000860
:1000B00095650008F3010008F3010008F30100084A
:1000C000F3010008F3010008F3010008F301000840
:1000D000F3010008F3010008F3010008F301000830
:1000E00025650008F3010008F3010008F30100088A
:1000F000F3010008F3010008F3010008F301000810
:10010000F3010008F3010008F3010008F3010008FF
:10011000F3010008F3010008F3010008F3010008EF
:10012000F3010008F3010008F3010008F3010008DF
:10013000F3010008F3010008F30100084D2D000849
:100140005D2D0008712D0008F3010008ED5900082D
:10015000F3010008F3010008F3010008F3010008AF
:10016000F3010008F3010008F3010008F30100089F
:10017000F3010008F3010008F3010008F30100088F
:10018000F3010008F3010008F3010008F30100087F
:10019000F3010008F3010008F3010008F30100086F
:1001A000F3010008F3010008F3010008F30100085F
:1001B000F3010008F3010008F3010008F30100084F
:1001C000F3010008F3010008F3010008F30100083F
:1001D000F3010008F3010008F3010008F30100082F
:1001E000C51500080000000000000000000000002D
:1001F00002E000F000F8FEE772B6374880F30888A6
:10020000364880F3098836483649086040F20000D5
:10021000CCF200004EF63471CEF200010860BFF35C
:100220004F8FBFF36F8F40F20000C0F2F0004EF628
:100230008851CEF200010860BFF34F8FBFF36F8F7C
:100240004FF00000E1EE100A4EF63C71CEF20001D4
:100250000860062080F31488BFF36F8F05F08EF8D6
:1002600005F072FF4FF055301F491B4A91423CBFC9
:1002700041F8040BFAE71D49184A91423CBF41F886
:10028000040BFAE71A491B4A1B4B9A423EBF51F82E
:10029000040B42F8040BF8E700201849184A914271
:1002A0003CBF41F8040BFAE705F06CF805F0A0FF3D
:1002B000144C154DAC4203DA54F8041B8847F9E797
:1002C00000F042F8114C124DAC4203DA54F8041B12
:1002D0008847F9E705F054B8000700200023002004
:1002E0000000000808ED00E00001002000070020E9
:1002F000986A000800230020B0230020B0230020CB
:1003000024670020E0010008E4010008E40100087F
:10031000E40100082DE9F04F2DED108AC1F80CD052
:10032000C3689D46BDEC108ABDE8F08F002383F3BF
:1003300011882846A047002004F028FBFEE704F0BF
:10034000A7FA00DFFEE70000F8B501F0A5F904F018
:10035000AFFF074604F0FEFF0546A8BB1F4B9F42B8
:1003600032D001339F4232D01D4B27F0FF029A4218
:1003700030D1F8B200F030FF2E4642F2107400F097
:1003800031FF08B10024264601F070FD20B10320A2
:1003900000F07AF80024264635B1124B9F4203D074
:1003A00004F0D0FF00242646002004F08BFF0EB19D
:1003B00000F080F801F0CCFA00F082FF204600F057
:1003C000DFF800F077F8F9E72E460024D7E7044677
:1003D0000126D4E7064641F28834D0E7010007B091
:1003E000000008B0263A09B008B501F027F9A0F1DD
:1003F00020035842584108BD07B541F212030221BB
:1004000001A8ADF8043001F037F903B05DF804FB42
:1004100038B5302383F31188174803680BB104F013
:1004200081FB164A144800234FF47A7104F070FBE4
:10043000002383F31188124C236813B12368013B16
:100440002360636813B16368013B63600D4D2B78D3
:1004500033B963687BB9022001F0E4F932236360A9
:100460002B78032B07D163682BB9022001F0DAF94E
:100470004FF47A73636038BDB02300201104000884
:10048000D0240020C8230020084B187003280CD863
:10049000DFE800F008050208022001F0B9B90220E7
:1004A00001F0ACB9024B00225A607047C82300200B
:1004B000D024002010B501F0D9FC30B1294B032223
:1004C0001A70294B00225A6010BD284B284A1C463E
:1004D00019680131F8D004339342F9D16268254B91
:1004E0009A42F1D9244B9B6803F1006303F58033F2
:1004F0009A42E9D204F0FAFE04F00CFF002001F069
:10050000E5F80220FFF7C0FF1C4B1A6C00221A64AA
:10051000196E1A66196E596C5A64596E5A665A6E7B
:100520005A6942F080025A615A6922F080025A6187
:100530005A691A6942F000521A611A6922F000528F
:100540001A611B6972B64FF0E0233021C3F8084DE1
:10055000D4E9003281F311889D4683F3088810475F
:10056000B2E700BFC8230020D0240020000001080B
:1005700020000108FFFF000800230020003802408F
:100580002DE9F04F93B0AC4B00902022FF210AA838
:100590009D6801F087F9A94A1378A3B9A8480121F9
:1005A00003601170302383F3118803680BB104F0EA
:1005B000B9FAA44AA24800234FF47A7104F0A8FAC9
:1005C000002383F31188009B13B19F4B009A1A609C
:1005D0009E4A009C1378032B1EBF002313709A4A77
:1005E0004FF0000A18BF5360D3465646D14601204B
:1005F00001F00EF924B1944B1B68002B00F015821A
:10060000002001F01BF80390039B002B01DA00F09F
:10061000A9FE039B002BEDDB012001F0EFF8039B0B
:10062000213B162BE3D801A252F823F089060008DB
:10063000B106000845070008EF050008EF050008AF
:10064000EF050008CF0700089F090008B908000857
:100650001B0900084309000869090008EF050008A4
:100660007B090008EF050008ED09000829070008CC
:10067000EF050008310A0008950600082907000860
:10068000EF0500081B0900080220FFF7ADFE002857
:1006900040F0F581009B0221BAF1000F08BF1C4613
:1006A00005A841F21233ADF8143000F0E5FF9EE7E3
:1006B0004FF47A7000F0C2FF071EEBDB0220FFF759
:1006C00093FE0028E6D0013F052F00F2DA81DFE833
:1006D00007F0030A0D10133605230593042105A81E
:1006E00000F0CAFF17E054480421F9E758480421F4
:1006F000F6E758480421F3E74FF01C08404600F0A5
:10070000E7FF08F104080590042105A800F0B4FFF4
:10071000B8F12C0FF2D1012000FA07F747EA0B0BD2
:100720005FFA8BFB4FF0000901F008F926B10BF0DE
:100730000B030B2B08BF0024FFF75EFE57E746486C
:100740000421CDE7002EA5D00BF00B030B2BA1D17C
:100750000220FFF749FE074600289BD0012000F049
:10076000B5FF0220FFF790FE00261FFA86F84046EC
:1007700000F0BCFF044690B10021404600F0CEFFDF
:1007800001360028F1D1BA46044641F21213022183
:1007900005A8ADF814303E4600F06EFF27E70120B3
:1007A000FFF772FE2546244B9B68AB4207D92846CB
:1007B00000F08EFF013040F067810435F3E7234BF2
:1007C00000251D70204BBA465D603E46ACE7002E0A
:1007D0003FF460AF0BF00B030B2B7FF45BAF0220F9
:1007E000FFF752FE322000F029FFB0F10008FFF6BB
:1007F00051AF18F003077FF44DAF0F4A926808EB32
:10080000050393423FF646AFB8F5807F3FF742AF0E
:10081000124B0193B84523DD4FF47A7000F00EFFC0
:100820000390039A002AFFF635AF019B039A03F861
:10083000012B0137EDE700BF00230020CC2400206E
:10084000B023002011040008D0240020C823002079
:1008500004230020082300200C230020CC230020A8
:10086000C820FFF7C1FD074600283FF413AF1F2D36
:1008700011D8C5F1200242450AAB25F0030028BF7C
:10088000424683490192184400F0E6FF019A8048ED
:10089000FF2101F007F84FEAA8037D490193C8F34F
:1008A0008702284601F006F8064600283FF46DAF9F
:1008B000019B05EB830537E70220FFF795FD002834
:1008C0003FF4E8AE00F04AFF00283FF4E3AE002713
:1008D000B846704B9B68BB4218D91F2F11D80A9B92
:1008E00001330ED027F0030312AA134453F8203C1F
:1008F00005934046042205A901F070FA04378046AA
:10090000E7E7384600F0E4FE0590F2E7CDF8148002
:10091000042105A800F0B0FE06E70023642104A826
:10092000049300F09FFE00287FF4B4AE0220FFF78E
:100930005BFD00283FF4AEAE049800F0F7FE059092
:10094000E6E70023642104A8049300F08BFE00284E
:100950007FF4A0AE0220FFF747FD00283FF49AAED7
:10096000049800F0F3FEEAE70220FFF73DFD0028BF
:100970003FF490AE00F002FFE1E70220FFF734FD04
:1009800000283FF487AE05A9142000F0FDFE0421E5
:100990000746049004A800F06FFE3946B9E73220FC
:1009A00000F04CFE071EFFF675AEBB077FF472AE7B
:1009B000384A926807EB090393423FF66BAE022078
:1009C000FFF712FD00283FF465AE27F003074F4400
:1009D000B9453FF4A9AE484600F07AFE04210590DF
:1009E00005A800F049FE09F10409F1E74FF47A7017
:1009F000FFF7FAFC00283FF44DAE00F0AFFE0028F0
:100A000044D00A9B01330BD008220AA9002000F031
:100A100051FF00283AD02022FF210AA800F042FF0F
:100A2000FFF7EAFC1C4803F0B7FF13B0BDE8F08FF6
:100A3000002E3FF42FAE0BF00B030B2B7FF42AAEEE
:100A40000023642105A8059300F00CFE074600284A
:100A50007FF420AE0220FFF7C7FC804600283FF459
:100A600019AEFFF7C9FC41F2883003F095FF0598F5
:100A700000F096FF464600F061FF3C46B7E50646AB
:100A800052E64FF0000905E6BA467EE637467CE6B8
:100A9000CC23002000230020A0860100094A13680F
:100AA00049F2690099B21B0C00FB01331360064B3D
:100AB000186844F2506182B2000C01FB0200186019
:100AC00080B27047182300201423002010B50021A5
:100AD0001022044600F0E6FE034B03CB2060616069
:100AE0001868A06010BD00BF107AFF1FF0B5ADF50B
:100AF0004D7D6AAC4FF4C47207460D462046002176
:100B000000F0D0FE02F06AF9264B4FF47A72B0FB87
:100B1000F2F0186093E80700022384E807000DF55F
:100B2000E5702382FFF7D2FF47F217031E492384A3
:100B300007A805F0CFFD0F2384F832310DF2DB2238
:100B400007AB0DF1240C1E4603CE664510605160C4
:100B5000334602F10802F6D130681060B188B379EB
:100B600093710BAE918020463146012200F01AFFAE
:100B700000230393AB7E029305F11903019380B226
:100B80000123CDE904600093E97E04A3D3E90023A7
:100B9000384602F039FD0DF54D7DF0BD9E6AC42149
:100BA000818A46EED8240020E46600082DE9F04151
:100BB0002C4C237ADAB080460D465BBB27A9284629
:100BC00001F016F80746002842D19DF89D60C82E16
:100BD0003ED801464FF4A662204600F063FE4FF473
:100BE0008073C4F8F8314FF40073C4F80C334FF439
:100BF0004073C4F8203432460DF19E0104F109001F
:100C000000F02AFE26449DF89C30777223720BB9BF
:100C1000EB7E23728122002106AC27A800F042FE61
:100C20000122214627A801F029F800230393AB7E77
:100C3000029305F1190380B201932823CDE9044002
:100C40000093E97E05A3D3E90023404602F0DCFCD3
:100C50005AB0BDE8F08100BFAFF300802641727248
:100C6000DF25D7B720350020F0B5254E4FF48A7523
:100C700005FB0065F1B096F8D83085F8DC3000242B
:100C8000D822214685F8E8403AA800F00BFE06F18C
:100C9000090000F0FFFDD5F8E4308DF8F000C2B295
:100CA00006AF06F109010DF1F100CDE93A3400F08B
:100CB000D3FD394601223AA801F016F880B2CDE9F9
:100CC000047008230127CDE9023706F1D803019308
:100CD00030230093317A0B4807A3D3E9002302F0B5
:100CE00093FCA04206DD02F079F8C5F8E000384632
:100CF00071B0F0BD2046FBE778F6339F93CACD8DE7
:100D000020350020F03400202DE9F04F274FDFF888
:100D1000A880274E87B0384602F0A2FC0346002880
:100D20003DD00024CDE90344ADF81440027B8DF89A
:100D3000142099684068029403AA03C21B681D4DE1
:100D400043F000430293A146A2462B68D3F810B0AB
:100D500002F046F810EB080241F100032846CDF8F6
:100D600000A002A9D84704F23A4440F674030028D0
:100D7000C8BF49F0010905F587559C4205F10805F2
:100D8000E3D1B9F1000F05D0384602F06DFC86F8CA
:100D900000A0C0E73378072B04D80133337007B0C5
:100DA000BDE8F08F014802F05FFCF8E7F034002066
:100DB000553A0020583A002040420F0070B50D46C9
:100DC00014461E4602F07CFB50B9022E10D1012CB5
:100DD0000ED112A3D3E90023C5E90023012007E0C7
:100DE000282C10D005D8012C09D0052C0FD00020BC
:100DF00070BD302CFBD10BA3D3E90023ECE70BA390
:100E0000D3E90023E8E70BA3D3E90023E4E70BA32E
:100E1000D3E90023E0E700BFAFF30080401DA1202D
:100E200026812A0B78F6339F93CACD8D9E6AC42102
:100E3000818A46EE26417272DF25D7B7F017304A15
:100E400039059E5638B505460E4C0021013500F097
:100E500065FCA4F82C55B4F82C0500F047FC78B1DB
:100E6000B4F82C0500F052FC014648B9B4F82C0542
:100E700000F054FCB4F82C350133A4F82C35EAE723
:100E800038BD00BF20350020F8B50E4C0E4F0226AD
:100E9000A4F5805343F8587C237E3BB965692DB196
:100EA000284601F061F8284601F09EF9204601F03D
:100EB0005BF8A4F58754012EA4F1080400D1F8BD15
:100EC0000126E5E7985B0020A06700082DE9F04FB8
:100ED0008FB000AF05460C4602F0F2FA00284BD165
:100EE000237E022B1BD1E38A012B18D101F076FF60
:100EF0000646FFF7D3FD03464FF4C870DFF8D482EF
:100F0000B3FBF0F206F5167602FB103316FA83F304
:100F1000C8F80030E37E33B9A74B00221A703C3783
:100F2000BD46BDE8F08F07F12401204600F014FE15
:100F30000028F4D107F11400FFF7C8FD97F8264008
:100F400007F11401224607F1270005F091FB002864
:100F5000E2D10F2C08D8984B1C70D8F80030A3F5BC
:100F60001673C8F80030DAE797F824100029D6D0B5
:100F7000284602F09DFAD2E7E38A282B33D010D816
:100F8000012B2BD0052BCAD1BFF34F8F8B498C4B34
:100F9000CA6802F4E0621343CB60BFF34F8F00BF17
:100FA000FDE7302BBBD1874EE17E327A9142B6D13C
:100FB000607E3146002291F8DC50854200F0AD8021
:100FC0000132042A01F58A71F5D1326840F6B83150
:100FD000FA328A4294BF32603160A0E72146284647
:100FE000FFF784FD9BE721462846FFF7DFFD96E7E4
:100FF000B2F8EC507B6005F103094FEA99094FEA1A
:101000008902D11DC908A8EBC1039D46EB4600210A
:10101000584600F047FC04F1EE012A463144584698
:1010200000F01AFC7B6813B9012000F04FFB96F822
:10103000D20000F05BFB044630B9307200F08EFB4A
:10104000204600F043FBB0E0D6F8D4203AB996F839
:10105000D200B6F82C25824201D8FFF7F3FED6F86D
:10106000D4202A44944208D296F8D200B6F82C250F
:101070000130824201D8FFF7E5FE70685FFA89F21D
:10108000594600F017FC08B9C54679E0726896F831
:10109000D2002A447260D6F8D42005EB0209C6F8C3
:1010A000D49000F023FB814509D396F8D220D6F8DE
:1010B000D4000132001B86F8D220C6F8D400FF2DE0
:1010C0000FD80024347200F049FB204600F0FEFAED
:1010D00000F0CCFE3C4B188108B9FFF7EBF9C54690
:1010E0001DE7BB6896F8D9000AFB0362FB68D2F8DB
:1010F000E41082F8E83001F58061C2F8E030C2F80F
:10110000E410FFF7B1FDFFF7FFFD96F8D92001329B
:1011100002F0030286F8D920B6E74FF48A7A0AFB78
:1011200002F505F1EA013144204600F011FEF860B5
:1011300000287FF4F4AE3544012285F8E82001F060
:101140004DFED5F8E020D6ED007ADFED206A801A5A
:10115000192838BF192040F6B832904228BF1046EF
:10116000B8EE677A07EE900AF8EEE77A67EEA67AAD
:10117000DFED176AE7EE267AFCEEE77AC6ED007A35
:1011800096F8D9307168BB600AFB03F4321992F803
:10119000E8505DB1D2F8E4308B42E8463FF428AF26
:1011A000002182F8E810C2F8E010C5467368064ACC
:1011B0009B0A01331381B2E6E934002000ED00E020
:1011C0000400FA0520350020D8240020CDCCCC3DE9
:1011D0006666663FEC340020014B1870704700BF14
:1011E000E424002030B54FF000542C4B22689A4282
:1011F00085B023D1637D0BB3294A2A481370237D20
:1012000003724FF48073C0F8F8314FF40073C0F8E4
:101210000C3300254FF44073C0F820342249C0F845
:10122000E450C922093000F017FB2046E02229468D
:1012300000F038FB0124204605B030BD04F094F8DE
:10124000044608B90024F6E7184A194D136C43F018
:1012500000731364AA6D174B9A42F3D12B6E013BB6
:101260007E2BEFD8144A07CA01AB83E80700184663
:10127000032100F0C9FD6B6D83424FF00003E1D103
:101280002A6D8A4201BFAB65054B2A6E1A7003BFF7
:101290000A4BEA6D1A601C46CDE700BF9AAD44C503
:1012A000E4240020203500201600002000380240F1
:1012B000006600405041A0B0586600401023002056
:1012C00037B500F0D3FD1D4D1D4C28810223216848
:1012D0001C486B71012201F001FC1B48216850F889
:1012E000E83F01225B68984700230193174B184998
:1012F00000931848184B4FF4805202F0B1F8174B86
:10130000197811B1134802F0D3F801F067FD0446D3
:10131000FFF7C4FB4FF4C873B0FBF3F202FB1303F7
:1013200004F5167010FA83F00D4B186004F012F8F3
:1013300008B10F232B8103B030BD00BFD82400209B
:1013400010230020583A0020584A0020BD0D000804
:10135000E8240020F0340020CD0E0008E424002012
:10136000EC3400202DE9F04F2DED028BDFF8508298
:1013700093B00BAF9FED838BFFF7C6FC00230A935E
:10138000ADF834300B937B600025844CDFF810A25D
:101390002E4601238DF81C3023688DED008B4FF015
:1013A000000BD3F808908DF81DB05B460DF11D02BF
:1013B00007A92046C8479DF81C90B9F1000F24D01A
:1013C000D8F8143083F48073C8F8143010225946CA
:1013D0000EA800F067FA236808AA5E690AA90DF151
:1013E0001E032046B04797E803000FAB83E80300D5
:1013F0009DF834308DF844300A9B0E930EA9DDE938
:101400000823504602F00EFB4E4605F23A4540F6E0
:10141000740304F587549D4204F10804B9D1002EE9
:10142000B2D15F4802F04CF8002840D15D4D01F088
:10143000D5FC2B6898423AD301F0D0FC0446FFF764
:101440002DFB4FF4C873B0FBF3F202FB130304F55A
:10145000167010FA83F02860534D8DF828602E78AE
:1014600016B901238DF82830C6F11004E4B20EA895
:10147000FFF72CFB062C28BF06240EAB2246991939
:101480000DF1290000F0E8F90AAB03931823029349
:101490000134464B0193E4B2012300934048049485
:1014A0003AA3D3E9002302F051F800232B7001F096
:1014B00095FC3F4A3F4C1368C31AB3F57A7F2FD38C
:1014C000106001F08DFC02460B46354802F0D6F85C
:1014D000334801F0F5FF18B3237A374D002B14BFC2
:1014E000032302236B7101F079FC0EAE4FF47A7383
:1014F0000122B0FBF3F031462860284600F004FBDF
:10150000182302932D4B019380B240F25513CDE97D
:101510000360009322481FA3D3E9002302F016F8CA
:10152000237A93B101F05AFC002506464FF48A77DE
:1015300094F8D900284400F0030007FB004393F817
:10154000E82072B10135042DF2D1C82003F024FA4D
:10155000237A002B7FF40DAF13B0BDEC028BBDE8F6
:10156000F08FD3F8E02042B12368FA2B38BFFA237A
:10157000B21A0533B2EB430FE4D3FFF775FB002833
:10158000E0D1E2E70000000000000000401DA120C3
:1015900026812A0BF1C6A7C1D068080F583A00204F
:1015A000F0340020EC340020E9340020E83400203E
:1015B000503A002020350020D8240020543A002042
:1015C0000008024008B5064800F0E0FF054800F0BA
:1015D000DDFFBDE80840044A0449002005F024B8B6
:1015E000583A0020404B0020645C0020890E00081F
:1015F00070B50F4B1B780133DBB2012B0C4611D8B1
:101600000C4D29684FF47A730E6AA2FB033201462F
:1016100022462846B047844204D1074B00221A7064
:10162000012070BD4FF4FA7003F0B6F90020F8E71E
:101630001C230020D85E0020545C002007B5002346
:10164000024601210DF107008DF80730FFF7D0FFAA
:1016500020B19DF8070003B05DF804FB4FF0FF30A8
:10166000F9E700000A4608B50421FFF7C1FF80F042
:101670000100C0B2404208BD30B4054C2368DD69AA
:10168000044B0A46AC460146204630BC604700BFCA
:10169000D85E0020A086010070B503F0ADFC094EB5
:1016A000094D3080002428683388834208D903F02C
:1016B0009DFC2B6804440133B4F5803F2B60F2D3CA
:1016C00070BD00BF565C0020285C002003F044BDC4
:1016D00000F1006000F580300068704700F10060A4
:1016E000920000F5803003F0CDBC0000054B1A6875
:1016F000054B1B889B1A834202D9104403F076BC29
:1017000000207047285C0020565C0020024B1B68BC
:10171000184403F073BC00BF285C0020024B1B6818
:10172000184403F083BC00BF285C002010F00303C2
:101730000AD1B0F5047F05D200F10050A0F51040A9
:10174000D0F80038184670470023FBE700F100503E
:10175000A0F51040D0F8100A70470000064991F833
:10176000243033B10023086A81F824300822FFF7BF
:10177000B5BF0120704700BF2C5C0020014B1868EA
:10178000704700BF002004E070B5194B1D68194B6D
:101790000138C5F30B0408442D0C04221E88A64210
:1017A0000BD15C680A46013C824213460FD214F901
:1017B000016F4EB102F8016BF6E7013A03F108033D
:1017C000ECD181420B4602D22C2203F8012B0A4AAB
:1017D00005241688AE4204D1984284BF967803F857
:1017E000016B013C02F10402F3D1581A70BD00BF35
:1017F000002004E03467000820670008022802BFC8
:10180000024B4FF480729A61704700BF000802409B
:10181000022802BF024B4FF080729A61704700BFEE
:1018200000080240022801BF024A536983F4807312
:10183000536170470008024070B504464FF47A7651
:101840004CB1412C254628BF412506FB05F003F08D
:10185000A3F8641BF4E770BD10B50023934203D0D6
:10186000CC5CC4540133F9E710BD000010B5013859
:1018700010F9013F3BB191F900409C4203D11AB1EC
:101880000131013AF4E71AB191F90020981A10BD1C
:101890001046FCE703460246D01A12F9011B002944
:1018A000FAD1704702440346934202D003F8011B69
:1018B000FAE770472DE9F8431F4D144695F82420A8
:1018C0000746884652BBDFF870909CB395F82430E9
:1018D0002BB92022FF2148462F62FFF7E3FF95F83E
:1018E0002400C0F10802A24228BF2246D6B24146D7
:1018F000920005EB8000FFF7AFFF95F82430A41BA2
:101900001E44F6B2082E17449044E4B285F82460D1
:10191000DBD1FFF723FF0028D7D108E02B6A03EBC8
:1019200082038342CFD0FFF719FF0028CBD10020DC
:10193000BDE8F8830120FBE72C5C0020024B1A78FD
:10194000024B1A70704700BF545C00201C2300201B
:1019500010B5104C104802F075FB21460E4802F0FD
:101960009DFB2468626DD2F8043843F00203C2F88C
:1019700004384FF47A70FFF75FFF0849204602F001
:1019800093FC626DD2F8043823F00203C2F80438E5
:1019900010BD00BF90680008D85E0020986800085D
:1019A000704700002DE9F3470D460446002190469C
:1019B000284640F27912FFF775FF234620220021C6
:1019C000284601F0D1FF231D02222021284601F0E4
:1019D000CBFF631D03222221284601F0C5FFA31D72
:1019E00003222521284601F0BFFF04F1080310223D
:1019F0002821284601F0B8FF04F1100308223821FD
:101A0000284601F0B1FF04F11103082240212846C5
:101A100001F0AAFF04F1120308224821284601F030
:101A2000A3FF04F1140320225021284601F09CFF5B
:101A300004F1180340227021284601F095FF04F1BB
:101A400020030822B021284601F08EFF04F1210373
:101A50000822B821284601F087FF04F12207C0269A
:101A60003B46314608222846083601F07DFFB6F590
:101A7000A07F07F10107F3D194F832308DF80730D9
:101A800031460DF107030822284601F06DFF0026BC
:101A900004F1330A9DF807304FEAC6099E4209F562
:101AA000A47720D394F83231502B28BF50238DF8DF
:101AB0000730B8F1000F08D139460DF107030722AE
:101AC000284601F051FF09F24F17002604F23314A3
:101AD0009DF807309E4207EBC6010DD30731C808B9
:101AE00002B0BDE8F0870AEB060308223946284613
:101AF00001F03AFF0136CDE7A3190822284601F08C
:101B000033FF0136E4E7000013B504460846002120
:101B100001602346C0F803102022019001F024FF49
:101B20000198231D0222202101F01EFF0198631D50
:101B30000322222101F018FF0198A31D0322252171
:101B400001F012FF019804F108031022282101F08E
:101B50000BFF072002B010BDF7B5047F05460E4607
:101B60002CB1838A122B02D9012003B0F0BD0023CF
:101B7000194607220096284601F0BAFD731C00930F
:101B8000012200230721284601F0B2FDD4B9B31C7D
:101B90000093052223460821284601F0A9FD0D24C3
:101BA000B378102BE0D83746B278BB1B934210D3E2
:101BB0002B7FA88A0734E408B3B9844294BF00207D
:101BC0000120D2E7AB8ADB00083BDB08B3700824B6
:101BD000E6E7FB1C0093214600230822284601F07B
:101BE00087FD08340137DFE7201A18BF0120BCE762
:101BF000F7B5047F05460E462CB1838ACA2B02D95D
:101C0000012003B0F0BD00231946009608222846A3
:101C100001F06EFD731CD4B90822009311462346CF
:101C2000284601F065FD10247378C82BE8D80123FD
:101C300072785F1C013B934210D32B7FA88A073434
:101C4000E408B3B9844294BF00200120D9E7AB8AED
:101C5000DB00083BDB0873700824E5E7F319009309
:101C6000214600230822284601F042FD08343B4665
:101C7000DEE7201A18BF0120C3E70000F7B50D46C4
:101C800004460021164628468122FFF70BFE234614
:101C900008220021284601F067FE94F901206378AC
:101CA000002AB8BF7F238DF807309EB90DF10703D6
:101CB00007220821284601F057FE0F27002602348C
:101CC0009DF807309E4207EBC60105D30731C808CF
:101CD00003B0F0BD0827F1E7A3190822284601F058
:101CE00043FE0136ECE70000F7B50E46054600213D
:101CF00014463046CE22FFF7D5FD2B462822002180
:101D0000304601F031FE2B7AC82B28BFC8238DF84E
:101D100007308CB90DF1070308222821304601F065
:101D200023FE30242F469DF807207B1B934205D3CA
:101D3000E01DC00803B0F0BD2824F3E707F1090354
:101D400021460822304601F00FFE08340137EAE749
:101D5000F7B5047F05460E4634B1838AB3F5827F1A
:101D600002D9012003B0F0BD00960123102200210A
:101D7000284601F0BDFCDCB9B31C009309222346C0
:101D80001021284601F0B4FC19247388B3F5807F34
:101D9000E7D837467288BB1B934210D32B7FA88AA3
:101DA0000734E408B3B9844294BF00200120D9E786
:101DB000AB8ADB00103BDB0873801024E5E73B1D9A
:101DC0000093214600230822284601F091FC0834A4
:101DD0000137DFE7201A18BF0120C3E730B5094DEE
:101DE0000A4491420DD011F8013B5840082340F3BA
:101DF0000004013B2C4013F0FF0384EA5000F6D1AD
:101E0000EFE730BD2083B8EDF7B54FF0FF33DFF8D3
:101E100054C0DFF854E000EB81011A4688421CD020
:101E200050F8044B019401AF042417F8015B82EAD7
:101E300005620825DB18164605F1FF355241002ED4
:101E4000BCBF83EA0C0382EA0E0215F0FF05F1D154
:101E5000013C14F0FF04E8D1E0E7D843D14303B0DC
:101E6000F0BD00BF9336EAA9EBE1F042F7B5384A7E
:101E7000106851686B4603C36A46364936480823E2
:101E800004F006FC0446002833D10A25334A1068C2
:101E900051686B4603C36A4631492F48082304F052
:101EA000F7FB0446002849D00369B3F5E02F45D875
:101EB000B0F8661041F2707291423FD1294A024453
:101EC00002F15C018B4239D35C3B234900209E1A0E
:101ED000FFF784FF3246074604F164010020FFF754
:101EE0007DFFA3689F4229D1E368984208BF00257F
:101EF00024E00369B3F5E02F27D8418B41F27072DB
:101F0000914220D1174A024402F110018B4218D3AA
:101F1000103B114900209D1AFFF760FF2A46064634
:101F200004F118010020FFF759FFA3689E4202D177
:101F3000E368984201D00D25A8E70025284603B0A4
:101F4000F0BD1025A2E70C25A0E70B259EE700BFFA
:101F500054670008DCFF0600000001085D67000808
:101F600090FF06000800FFF710B5037C044613B984
:101F7000006804F075FB204610BD00000023BFF38D
:101F80005B8FC360BFF35B8FBFF35B8F8360BFF377
:101F90005B8F7047BFF35B8F0068BFF35B8F704749
:101FA00070B505460C30FFF7F5FF05F1080604464D
:101FB0003046FFF7EFFFA04206D930466D68FFF7C5
:101FC000E9FF2544281A70BD3046FFF7E3FF201AC9
:101FD000F9E7000070B50546406898B105F10800C2
:101FE000FFF7D8FF05F10C0604463046FFF7D2FF95
:101FF0008442304694BF6D680025FFF7CBFF013C5B
:102000002C44201A70BD000038B50C460546FFF779
:10201000C7FFA04210D305F10800FFF7BBFF04443F
:102020006868B4FBF0F100FB1144BFF35B8F012043
:10203000AC60BFF35B8F38BD0020FCE72DE9F041B9
:10204000144607460D46FFF7C5FF844228BF0446E5
:10205000D4B1B84658F80C6B4046FFF79BFF3044AC
:10206000286040467E68FFF795FF331A9C4203D8EC
:102070006C600120BDE8F0816B60A41B3B68AB6025
:102080002044E8600220F5E72046F3E738B50C4627
:102090000546FFF79FFFA04210D305F10C00FFF7A4
:1020A00079FF04446868B4FBF0F100FB1144BFF30E
:1020B0005B8F0120EC60BFF35B8F38BD0020FCE735
:1020C0002DE9FF41884669460746FFF7B7FF6C4692
:1020D00006B204EBC6060025B44209D06268206847
:1020E00008EB0501FFF7B8FB636808341D44F3E70C
:1020F00029463846FFF7CAFF284604B0BDE8F081FC
:10210000F8B505460C300F46FFF744FF05F1080609
:1021100004463046FFF73EFFA042304688BF6C6859
:10212000FFF738FF201A386020B130462C68FFF7DF
:1021300031FF2044F8BD000073B5144606460D4635
:10214000FFF72EFF844228BF04460190DCB101A9AD
:102150003046FFF7D5FF019B33B93268C5E902333A
:10216000C5E9002401200CE09C4238BF019428609E
:10217000019868608442F5D93368AB60241AEC603A
:10218000022002B070BD2046FBE700002DE9FF41B0
:102190000F466946FFF7D0FF6C4600B204EBC0055E
:1021A0000026AC4209D0D4F8048054F8081BB819B2
:1021B0004246FFF751FB4644F3E7304604B0BDE822
:1021C000F081000038B50546FFF7E0FF0446014600
:1021D0002846FFF719FF204638BD0000012188423C
:1021E00038BF084604F026BA08B104F039BA70477F
:1021F00010B4026854681A4623465DF8044B184729
:102200000020704700207047704700000020704792
:102210000E20704700F5805090F8D800C0F34000C1
:102220007047000000F5805090F9E0007047000012
:1022300000F58050C0F8DC1001207047F7B50C683D
:10224000BDF8207014F0005473D10D7B082D70D8A8
:10225000302585F31188456AAE6876010CD4AC68E8
:10226000240108D4AC6814F0805460D184F3118840
:10227000204603B0F0BD01240E6804F1180C002EB6
:10228000B8BFF6004FEA0C1CB4BF46F00406760552
:1022900045F80C600E680FFA84FC16F0804F18BFEA
:1022A00005EB0C1E05EB0C1C1EBFDEF8806146F032
:1022B0000206CEF880610E7BCCF8846105EB041534
:1022C0008E68C5F88C614E68C5F88861DCF880516D
:1022D00045F00105CCF8805141F2780500EB441C33
:1022E000660105EB4414AC440444CCE900230D46DC
:1022F000083401F10C0C55F804EB44F804EB654587
:10230000F9D12D882580841904F5805407F0030540
:1023100094F8946026F00B06354384F8945000241A
:1023200084F31188009700F0A3FD0120A1E70224A7
:10233000A2E74FF0FF309CE713B500F58054019100
:10234000E06EFFF747FE1F280AD90199E06E2022B0
:10235000FFF7B6FEA0F120035842584102B010BD6D
:102360000020FBE708B5302383F3118800F5805087
:10237000C06EFFF703FE002383F3118808BD000041
:1023800000220260828142608260704710B50022A4
:102390000023C0E900230023044603810C30FFF72B
:1023A000EFFF204610BD0000F0B5054600F5805057
:1023B0000C4690F8D83013F0040FC3F3800108BF27
:1023C000114661F3820380F8D83005EB441303F51E
:1023D0008453103389B01B79D8074FEA44162FD5A0
:1023E00082B319072ED46846FFF7D0FF05EB4413DC
:1023F00003F5845303AA03F10807186859681446C3
:1024000003C40833BB422246F7D1186820609B887A
:10241000A380DDE90E23CDE900230123ADF80830C8
:102420002B6869461B6C28469847354405F584554A
:1024300010352B791A075CBF43F008032B7101E0BC
:10244000002AF2D109B0F0BD2DE9F0479A4688B0D4
:10245000074688469146302383F3118807F5805458
:102460006846FFF793FFE06EFFF79AFD1F282AD911
:10247000E06E20226946FFF7A5FE202823D103AD98
:10248000444605AB2E4603CE9E4220606160354631
:1024900004F10804F6D130682060B388A380DDE938
:1024A0000023C9E90023BDF80830AAF80030002352
:1024B00083F3118853464A464146384608B0BDE882
:1024C000F04700F099BC002080F3118808B0BDE807
:1024D000F08700002DE9F84F182204460F4604301B
:1024E0000021FFF7DFF92046254B40F8283BFFF796
:1024F00047FF04F13800FFF749FF04F1580804F5DD
:1025000082554646183530462036FFF73FFFAE422B
:10251000F9D104F580554FF480534FF00009C5E917
:102520001739C5F858800123EE6604F5875804F57D
:102530008456C5F8649085F8683085F87030183690
:1025400008F118084FF0000A4FF0000B46E908ABFD
:10255000A6F11800FFF714FF203646F8289C4645E0
:10256000F4D1012F85F8E07002D9064800F030FC64
:10257000054B53F8273063622046BDE8F88F00BF53
:10258000A0670008686700088467000810B5044B5E
:10259000197804464A1C1A70FFF79CFF204610BDAC
:1025A000605C00202DE9F047002950D0294B2A4FCC
:1025B000B7FBF1F599428CBF0A231123581EB5FBD6
:1025C000F3FC03FB1C53C4B22BB102280346F5D81D
:1025D0000020BDE8F0870CF1FF36B6F5806FF7D22A
:1025E000C4EBC40E0EF103034FEAE309C3F3C703C0
:1025F000A4EB030809F1010A4FF47A755FFA88F039
:1026000009FB05555AFA88F8B5FBF8F5B5F5617F71
:10261000C1BF0EF1FF33C3F3C703E01AC0B25C1CA5
:1026200050FA84F40CFB04F4B7FBF4F4A142CFD1CC
:10263000013BDBB20F2BCBD80138C0B20728C7D87B
:102640000021107116809170D3700120C1E70846F7
:10265000BFE700BF3F420F0080DE800270B5054635
:102660000E464FF47A746B6A5B6803F00103B34261
:1026700007D04FF47A7002F08FF9013CF3D1204675
:1026800070BD0120FCE7000070B5426A936913F049
:10269000700F17D000230C4D936141F2900400EBB2
:1026A0004312224411794E0709D5890707D5416A9B
:1026B00055F823608E60117941F0040111710133E6
:1026C000032BECD170BD00BF8C67000873B51D46AD
:1026D000436A16469A68D207044609D59A680121CA
:1026E0009960C2F34002CDE900650021FFF75CFE6E
:1026F000636A9A68D1050BD59A684FF48071996026
:10270000C2F34022CDE9006501212046FFF74CFECF
:10271000636A9A68D2030BD59A684FF48031996046
:10272000C2F34042CDE9006502212046FFF73CFE9E
:1027300004F58053D3F8DC0010B103681B69984797
:10274000204602B0BDE87040FFF79EBF0C4B10B5AD
:102750001C561B5C012B11D800F042FB50EA010310
:10276000024602D0421E61F10001064B53F82400DC
:1027700020B1BDE810400B46FFF7A8BF10BD00BF59
:1027800080670008585C0020F8B50446466A0029B6
:1027900077D106F10C073868800775D006EB011574
:1027A0003868D5F8B00110F0040FD5F8B0011ABFA1
:1027B000C00840F00040400DA062D5F8B0C11CF048
:1027C000020F1CBF40F08040A062D5F8B40106EBB8
:1027D000011100F00F0084F83400D1F8B80184F83A
:1027E0002C00D1F8B801000A84F82D00D1F8B80106
:1027F000000C84F82E00D1F8B801000E84F82F00E8
:10280000D1F8BC0184F83000D1F8BC01000A84F88A
:102810003100D1F8BC01000C84F83200D1F8BC11B1
:10282000090E84F833103821396004F1440004F1B2
:10283000280104F1340551F8046B40F8046BA942F7
:10284000F9D109880180C4E90E2321460023A4F8A8
:10285000403051F8383B20461B6C984704F58053B4
:1028600093F8D820D3F8DC0042F0040283F8D82093
:1028700010B103681B6998472046BDE8F840FFF790
:1028800003BF06F1100786E7F8BD00000D4B70B5D9
:102890001D561B5C012B0C4612D800F0A1FA024613
:1028A0000B4652EA030102D0013A63F100030649E4
:1028B00051F8250020B12146BDE87040FFF764BF04
:1028C00070BD00BF80670008585C0020F0B5302163
:1028D00081F31188DFF848E000F5835118310024B6
:1028E00041F2900C00EB441565442E7977070ED425
:1028F000F6060CD5D1E9007697429E4107D2466A8A
:102900005EF82470B7602E7946F004062E7101340B
:10291000032C01F12001E5D1002383F31188F0BDE0
:102920008C67000808B5302383F31188FFF7ACFEED
:10293000002383F3118808BD2DE9F041436A044662
:10294000986800F0E050B0F1E05F0E4622D0F8B198
:10295000302383F31188002504F5845741F2900851
:1029600004EB451343441B791A0706D50135032DA3
:1029700007F12007F4D1012007E05B07F6D43946C0
:10298000304600F0C7FA0028F0D1002383F3118805
:10299000BDE8F0810120FBE708B5302383F31188FF
:1029A00000F58050C06EFFF7FBFA002383F3118817
:1029B00043090CBF0120002008BD0000F8B51D46EA
:1029C000002313700F4606461446FFF7E5FF80F01C
:1029D0000100387025B129463046FFF7ADFF207061
:1029E000F8BD00002DE9B8410C4615461F4680464B
:1029F00000F0F6F90B462178024609B9287850B163
:102A00004046FFF763FFFFF78DFF3B462A4621460E
:102A1000FFF7D4FF0120BDE8B881000038B53023AE
:102A200083F3118800F580542A4D94F8E030EB5C74
:102A3000E3B1012B28D0002383F3118894F8D83018
:102A4000DB0712D489B1302383F3118894F8E03086
:102A5000EB5C33B3012B31D094F8D83043F0010351
:102A600084F8D830002383F3118838BD1A4B1A6CD0
:102A700042F000721A641A6A42F000721A621A6A0C
:102A800022F000721A62D6E7134B1A6C42F0806291
:102A90001A641A6A42F080621A621A6A22F080622C
:102AA000F0E70321132001F03DFA0321142001F087
:102AB00039FA0321152001F035FACDE703213F2033
:102AC00001F030FA0321402001F02CFA03214120CB
:102AD000F1E700BF7C670008003802402DE9F047AD
:102AE00000F5805588B095F8E030022B0446884602
:102AF000164600F28280864F57F823200AB947F81D
:102B00002300D7F800A0C4F81C8084F82060BAF134
:102B1000000F64D095F8E030012B70D001212046E1
:102B2000FFF77CFF302383F31188626A136823F078
:102B300002031360626A136843F001031360636A5F
:102B400000275F6187F3118801212046FFF786FD8A
:102B5000002800F09580E86EFFF710FA04F583591D
:102B6000BA4609F11809202200216846FEF79AFEAC
:102B700002A8FFF705FCCDF818A06A4609EB070389
:102B80000DF1180E9446BCE80300F4451860596036
:102B9000624603F10803F5D1DCF800001860203725
:102BA0009CF804201A71602FDDD195F8D8306FF3AE
:102BB0008203002785F8D8306A4641462046ADF8A2
:102BC0000070ADF802708DF80470FFF7EBFC636ADB
:102BD00048BB4FF400421A6008B0BDE8F08741F2EC
:102BE000E800FFF7FBFA814610B15146FFF772FC8F
:102BF000C7F80090B9F1000F8CD10020ECE73868DD
:102C000003681B6B98470146002887D13868FFF797
:102C100005FF3868036832465B68414698470028DC
:102C20007FF47CAFE9E761221A609DF802309DF8DD
:102C300003201B06120402F4702203F040731343B6
:102C4000BDF80020C2F3090213439DF804201205C9
:102C5000022E02F4E0020CBF4FF0004100211343AA
:102C6000626A0B43D361636A13225A61626A136812
:102C700023F00103136039462046FFF7EFFC08B943
:102C8000636AA6E795F8E030002B39D1616AD1F884
:102C9000002242F00102C1F80022616AD1F800224C
:102CA00022F47C5222F00E02C1F80022616AD1F8AF
:102CB000002242F46062C1F80022626AC2F8143253
:102CC000626AC2F80432626A6FF07841C2F80C128C
:102CD000626AC2F84032626AC2F84432626AC2F87A
:102CE000B032626AC2F8B432636A44F20102C3F8D5
:102CF0001C22626AD2F8003223F00103C2F80032CB
:102D000095F8D83043F0020385F8D83064E700BF67
:102D1000585C002008B50020FFF718FDBDE808400A
:102D200001F0D6B808B500210846FFF7AFFDBDE8B1
:102D3000084001F0CDB8000008B501210020FFF7E0
:102D4000A5FDBDE8084001F0C3B8000008B50120AA
:102D5000FFF7FCFCBDE8084001F0BAB808B5002157
:102D60000120FFF793FDBDE8084001F0B1B8000075
:102D700008B501210846FFF789FDBDE8084001F0CC
:102D8000A7B8000000B59BB0EFF309816822684640
:102D9000FEF762FDEFF30583014B9B6BFEE700BF7F
:102DA00000ED00E008B5FFF7EDFF000000B59BB0B7
:102DB000EFF3098168226846FEF74EFDEFF30583C5
:102DC000014B5B6BFEE700BF00ED00E0FEE700009B
:102DD0000FB408B5029801F085FDFEE702F006BACF
:102DE00002F0E8B90139C9B202299EBF00EBC10067
:102DF0000023C0E901337047F8B51B885B0705461F
:102E00000E4615D4044600F11807BC4210D0636882
:102E100053B12B682846DB6B9847A368C1B2324692
:102E2000606898470834F0E7A368002BF1D1F9E710
:102E30000120F8BD73B56C4684E806000146002207
:102E40004E68D5B26EB98E685EB900EBC200021D45
:102E500094E80300013582E803001D70012002B0F0
:102E600070BD0132032A01F10801E9D10020F6E723
:102E70002DE9F04F89B00446BDF848700E4605466E
:102E800000F118084FF0000907F004074FF0000A9E
:102E90004FF0000BA84538D06B680BB9AB684BB14D
:102EA00057B923682046DB6B9847AB68C1B23246FE
:102EB000686898470835EDE7B9F1000FFAD1CDE918
:102EC00000ABADF80890334603AA06F1080E186867
:102ED00059689446ACE80300083373456246F6D15E
:102EE0001868CCF800009B88ACF80430FFF778FF36
:102EF0000423ADF808302368CDE900011B6C694656
:102F0000204698474FF00109D4E7012009B0BDE8F9
:102F1000F08F000030B503680968DD0FB5EBD17F95
:102F200023F0604421F060424FEAD1700BD0002BB7
:102F3000B8BFA40C0029B8BF920C944202D034BF91
:102F40000120002030BD944205D1C1F38070C3F34D
:102F500080738342F6D194422CBF00200120F1E718
:102F60002DE9F041456A15B94162BDE8F0814B6831
:102F700023F06047C3F38A464FEAD37EC3F38078D9
:102F800016EA230638BF3E46AC462B465A68BEEBCF
:102F9000D27F22F060440AD0002A18DAA40CB4428E
:102FA00017D19D420FD10D60DEE71346EEE7A74231
:102FB00007D102F08044C2F3807242450BD054B175
:102FC000EFE708D2EDE7CCF800100B60CDE7B44294
:102FD00001D0B442E5D81A689C46002AE5D11960B0
:102FE000C3E700002DE9F047089D01F007044FEA10
:102FF000D508224405F0070500EBD1004FF47F49C6
:10300000944201D1BDE8F08704F0070705F0070AF4
:1030100057453E4638BF5646C6F10806111B8E423C
:1030200028BF0E46E10808EBD50E415C13F80EC030
:10303000B94029FA06F721FA0AF1FFB28CEA010138
:1030400047FA0AF739408CEA010C03F80EC0344401
:103050003544D5E780EA0120082341F2210201B27C
:103060004000002980B203F1FF33B8BF504013F095
:10307000FF03F4D17047000038B50C468D18A54207
:1030800000D138BD14F8011BFFF7E4FFF7E700009B
:1030900042684AB1136843604389818901339BB216
:1030A0009942438138BF83811046704770B588B01C
:1030B000202204460D4668460021FEF7F3FB204619
:1030C0000495FFF7E5FF024658B16B46054608AE8A
:1030D0001C4603CCB44228606960234605F108050C
:1030E000F6D1104608B070BD082817D909280CD0B1
:1030F0000A280CD00B280CD00C280CD00D280CD092
:103100000E2814BF4020302070470C20704710203C
:103110007047142070471820704720207047000027
:10312000082817D90C280CD910280CD914280CD928
:1031300018280CD920280CD930288CBF0F200E203D
:103140007047092070470A2070470B2070470C20F9
:1031500070470D20704700002DE9F843078C072FBA
:1031600004461ED9D0E9029800254FF6FF73C5F139
:103170002006A5F1200029FA05F108FA06F628FA3A
:1031800000F031430143C9B21846FFF763FF083529
:10319000402D0346EBD1E1693A46BDE8F843FFF71D
:1031A0006BBF4FF6FF70BDE8F883000010B54B68A9
:1031B00023B9CA8A63F30902CA8210BD04691A6876
:1031C0001C600361C38A013BC3824A60EFE70000D1
:1031D0002DE9F84F1D46CB8A0F46C3F30901052997
:1031E000814692460B4630D00020AAB207F11A045D
:1031F0009EB2042E1FFA80F80FD8904503F1010308
:1032000006D3FB8A0A4462F30903FB8201201AE019
:103210001AF80060E6540130EAE79045F1D2A1F1D6
:10322000050B1C237C68BBFBF3F203FB12BB1FFAEC
:103230008BF6002C45D14846FFF72AFF044638B9E3
:1032400078606FF00200BDE8F88F4FF00008E6E705
:10325000002606607860ADB24FF0000B454510D9EE
:103260000AEB0803221D13F8011B9155B1B208F1B6
:1032700001081B291FFA88F82BD0454506F10106E5
:10328000F1D8FB8AC3F30902154465F30903BCE7CF
:10329000013292B21C462368002BF9D16B1F0B44FC
:1032A0001C21B3FBF1F301339BB29A42D3D2BBF1A1
:1032B000000FD0D14846FFF7EBFE20B9C4F800B0AC
:1032C000BFE70122E7E7C0F800B05E462060044691
:1032D000C1E74545D5D94846FFF7DAFE08B9206071
:1032E000AFE7C0F800B0002620600446B6E7000053
:1032F0002DE9F04F2DED028B1C4683B05B690192E6
:1033000007468846002B00F0A780238C2BB1E2698A
:10331000002A00F0A180072B35D807F10C00FFF739
:10332000B7FE054638B96FF00205284603B0BDEC7C
:10333000028BBDE8F08F14220021FEF7B3FA228C35
:10334000E16905F10800FEF787FA208C013080B2B0
:10335000FFF7E6FEFFF7C8FE013880B22084013097
:1033600028746369228C1B782A4403F01F0363F0DE
:103370003F0348F000411372384669602946FFF761
:10338000EFFD0125D1E702339BB20722C18A063344
:10339000B3FBF2F3828A521A9BB292B29342C2D822
:1033A00000F10C034FF0000908EE103A4FF0800ACC
:1033B0004E464D4618EE100AFFF76AFE8346002877
:1033C000B1D014220021FEF76DFA002E3AD1019BF4
:1033D000ABF8083002220BF1080E1FFA82FC0CF148
:1033E0000100BCF1060F218C80B201D88E422BD394
:1033F000FFF796FEFFF778FE62691278013802F057
:103400001F028E4208BF4FF0400A42EA49121BFADF
:1034100080F14AEA020A013048F0004281F808A02F
:103420008BF81000CBF8042059463846FFF798FD7A
:10343000238C0135B3422DB289F001094FF0000A07
:10344000B8D172E70022C6E7E169895D0EF8021083
:103450000136B6B20132C0E76FF0010565E7000042
:10346000F8B515460E463022002104461F46FEF7E9
:1034700019FA069B6360B5F5001F079BA76034BF70
:103480006A094FF6FF72A36297B2E66104F1100079
:1034900000239A4206D800230360A782E382238395
:1034A000E360F8BD0660013330462036F1E70000E6
:1034B00003781BB94BB2002BC8BF017070470000E6
:1034C00000787047F8B50C46C969074611B9238CD6
:1034D000002B37D1257E1F2D34D8387828BB228C7D
:1034E000072A2CD8268A36F003032BD14FF6FF701B
:1034F000FFF7C2FD20F001003102400441EA0561FE
:10350000400C41EA40254FF6FF72234629463846D3
:10351000FFF7EEFE002807DD626913780133DBB2A6
:103520001F2B88BF00231370F8BD218A2D0645EAA2
:10353000012505432046FFF70FFE0246E5E76FF041
:103540000300F1E76FF00100EEE7000070B58AB00C
:10355000044616460021282268461D46FEF7A2F9B9
:10356000BDF83830ADF810300F9B05939DF8403012
:103570008DF81830119B07936946BDF84830ADF8B7
:1035800020302046CDE90265FFF79CFF0AB070BDF0
:103590002DE9F041D36905460C4616460BB9138C4C
:1035A0005BBB377E1F2F28D895F80080B8F1000F3D
:1035B00026D03046FFF7D0FD3378210241EAC331EF
:1035C00041EA0801338A41EA076141EA03410246C0
:1035D000334641F080012846FFF78AFE00280ADDC5
:1035E0003378012B07D1726913780133DBB21F2BBB
:1035F00088BF00231370BDE8F0816FF00100FAE787
:103600006FF00300F7E70000F0B58BB004460D46FD
:1036100017460021282268461E46FEF743F99DF80A
:103620004C305A1E534253418DF800309DF84030C3
:10363000ADF81030119B05939DF848308DF8183087
:10364000149B07936A46BDF85430ADF820302946E4
:103650002046CDE90276FFF79BFF0BB0F0BD0000DE
:10366000406A00B104307047436A1A6842620269D6
:103670001A600361C38A013BC38270472DE9F041A0
:10368000D0F82080194E14461D464146002709B93E
:10369000BDE8F081D1E90223A21A65EB030396424B
:1036A00077EB03031ED2036A8B420DD1FFF77EFD39
:1036B000036A1B68036203690B60C38A0161016AC4
:1036C000013BC3828846E2E7FFF770FD0B68C8F84C
:1036D000003003690B60C38A0161013BC382D8F8E3
:1036E0000010D4E788460968D1E700BF80841E0037
:1036F0002DE9F04F8BB00D46DDF8509014469B46F7
:103700008046002800F01981B9F1000F00F0158102
:10371000531E3F2B00F21181012A03D1BBF1000F90
:1037200040F00B810023CDE90833B8F81430B5EB35
:10373000C30F4FEAC30703D300200BB0BDE8F08FDF
:103740002B199F42D8F80C303ABF7F1BFFB2274697
:103750001BB9D8F81030002B7AD0272D4ED8C5F1E0
:103760002806B7424FF000032CBFF6B23E46009346
:103770002946D8F8080008AB3246FFF733FCA7EB20
:10378000060A35445FFA8AFAB8F8143003F1005398
:10379000053BDB000493D8F80C3003932821039BEE
:1037A00013B1BAF1000F2CD1D8F8100040B1BAF122
:1037B000000F05D0009608AB5246691AFFF712FCBD
:1037C00038B2002FB8D066070AD00AAB03EBD40199
:1037D000624211F8083C02F00702134101F8083C6C
:1037E000082C3CD9102C40F2B580202C40F2B78038
:1037F000BBF1000F00F09C80082334E0BA4600269D
:10380000C2E7049BE02B28BFE02306930B44AB42A6
:10381000059314D95A1B03980096924534BF52461B
:10382000D2B2691A08AB04300792FFF7DBFB079AA4
:103830001644AAEB020A1544F6B25FFA8AFA049B10
:10384000069A05999B1A0493039B1B680393A6E7AA
:103850000093D8F8080008AB3A462946AEE7BBF11A
:10386000000F13D00123B4EBC30F6CD0082C12D877
:103870009DF82030621E23FA02F2D50706D54FF0DC
:10388000FF3202FA04F423438DF820309DF82030F3
:1038900089F8003051E7102C12D8BDF82030621E94
:1038A00023FA02F2D10706D54FF0FF3202FA04F4F0
:1038B0002343ADF82030BDF82030A9F800303CE7B4
:1038C000202C0FD80899631E21FA03F3DA0705D5D7
:1038D0004FF0FF3202FA04F40C430894089BC9F835
:1038E00000302AE7402C2BD0DDE90865611EC4F1C9
:1038F0002102A4F1210326FA01F105FA02F225FAC8
:1039000003F311431943CB0712D50122A4F120037D
:10391000C4F1200102FA03F322FA01F1A24052425B
:1039200043EA010363EB430332432B43CDE908230E
:10393000DDE90823C9E90023FFE66FF00100FCE69A
:103940006FF00800F9E6082CA0D9102CB3D9202C70
:10395000EED8C3E7BBF1000FADD0022383E7BBF184
:10396000000FBBD004237EE730B5012A144638BFD0
:103970000124402C85B028BF40240025012ACDE930
:10398000025518D81B788DF8083063070AD004ABAD
:1039900003EBD405624215F8083C02F0070293409D
:1039A00005F8083C009103462246002102A8FFF7D3
:1039B00019FB05B030BD082AE4D9102A03D81B88AA
:1039C000ADF80830E1E7202A8DBFD3E900231B685A
:1039D0000293CDE90223D8E710B5CB681BB98B6001
:1039E0000B618B8210BD04691A681C600361C38A75
:1039F000013BC382CA60F0E703064CBFC0F3C0308E
:103A00000220704708B50246FFF7F6FF022806D1EC
:103A10005306C2F30F2001D100F0030008BDC2F32A
:103A20000740FBE72DE9F04F93B0CDE903230A6887
:103A300004461046FFF7E0FF022814BFC2F3062633
:103A40000026002A0D46824680F2F78112F0C04916
:103A500040F0F381097B002900F0EF81022803D0B8
:103A60002378B34240F0EC81C2F30463069310461E
:103A700002F07F030593FFF7C5FF059B29444FEA3A
:103A8000834848EA0A4848EA4668CE78002300227C
:103A9000CDE90823F309834648EA0008029367D07A
:103AA000059B009302466768534608A92046B8471D
:103AB000002800F0C881276A4FB9414604F10C0084
:103AC000FFF7F4FA074690B96FF0020054E03B6943
:103AD00098450DD03F68002FF9D1414604F10C0004
:103AE000FFF7E4FA07460028EED0236A3B6027621E
:103AF00097F817C006F01F08CCF3840CACEB080055
:103B00001FFA80FE0028B8BF0EF12000A8EB0C03BE
:103B10001FFA83FED7E90221B8BF00B2002B07933A
:103B2000BEBF0EF120031BB2079352EA010338D047
:103B3000039BDFF824E39A1A049B4FF0000C63EB1D
:103B4000010196457CEB01032BD36B7B97F81AE0C0
:103B5000734519D1029B002B78D0012821DC7868AD
:103B6000F8B9DFF8F0C2944570EB010316D337E0E3
:103B7000276A27B96FF00C0013B0BDE8F08F3B69DE
:103B80009845B5D03F68F4E7B24890427CEB01031A
:103B900001D30020F0E7029B002BFAD0079B0F2BEC
:103BA00017DCFA7DB30002F0030203F07C03134339
:103BB000FB7539462046FFF7F9FA6B7BBB76029B13
:103BC0003BB9FB7DC3F38402013262F38603FB75CC
:103BD000D0E76A7BBB7E9A42DBD1029B002B35D0BB
:103BE000B309022B32D0039BBB60049BFB60142201
:103BF00000210DA8FDF756FE039B0A93049B0B932F
:103C00002B1D0C932B7BADF83EB0013BDBB2ADF826
:103C10003C30069B8DF84230059B8DF8433094F87C
:103C20002C308DF840A083F001038DF844308DF8DE
:103C30004180A3680AA920469847FB7DC3F384030B
:103C4000013303F01F039B02FB82A2E7FB7DC6F357
:103C50004012B2EBD31F40F0F980C3F38403434515
:103C600040F0FC80029A2B7BB609002A52D016F055
:103C7000010661D1032B40F2F480039BBB60049BDF
:103C8000FB60FB8A66F30903FB822B7BAE1D033BC3
:103C9000DBB23246394604F10C00FFF799FA0028EE
:103CA0000CDA39462046FFF781FAFB7DC3F3840323
:103CB000013303F01F039B02FB8205E7DDE9088463
:103CC000AB883B834FF6FF73C9F12000A9F12002B6
:103CD00028FA09F104FA00F0014324FA02F2114330
:103CE0001846C9B2FFF7B6F909F10809B9F1400F52
:103CF0000346E9D1B8822A7B033AD2B23146FFF7B4
:103D0000BBF9FB7DB882DA43C2F3C01262F3C7137A
:103D1000FB753EE786B92E1D013BDBB232463946C4
:103D200004F10C00FFF754FA0028BADB2A7BB88AAA
:103D3000013AD2B23146E2E7F98AC1F30901013B07
:103D40000429DAB25BD8281D002307F11B069A422A
:103D500008D910F801CB06F801C00131013305295B
:103D6000DBB2F4D103990A9104990B91934207F1C4
:103D70001B010C9138BF043379680D9134BF55FA9B
:103D800083F300230E93FB8AADF83EB0C3F309031F
:103D90001A44069B8DF84230059B8DF8433094F809
:103DA0002C30ADF83C2083F001038DF84430002323
:103DB0008DF840A08DF841807B602A7BB88A013A5B
:103DC000291DFFF759F93B8BB882834203D1A368C1
:103DD0000AA92046984720460AA9FFF7FDFDFB7D6A
:103DE000BA8AC3F38403013303F01F039B02FB82EF
:103DF0003B8B9A420CBF00206FF01000BCE67B6842
:103E0000002BAFD0052001E01C3033461E68002E89
:103E1000FAD1091A081D2E1D184401EB090CBCF13A
:103E20001B0F5FFA89F39DD89A429BD916F8013B84
:103E300000F8013B09F10109EFE76FF009009BE68B
:103E40006FF00A0098E66FF00B0095E66FF00D003A
:103E500092E600BF40420F0080841E006FF00E000B
:103E60008AE66FF00F0087E6EFF3098305494A6B96
:103E700022F001024A63683383F30988002383F345
:103E80001188704700EF00E0302080F3118862B69F
:103E90000C4B0D4AD96821F4E0610904090C0A436E
:103EA000DA60D3F8FC20094942F08072C3F8FC20A4
:103EB0000A6842F001020A602022DA7783F82200C1
:103EC000704700BF00ED00E00003FA05001000E0BD
:103ED00010B5302383F311880E4B5B6813F4006335
:103EE00014D0F1EE103AEFF30984683C4FF0807380
:103EF000E361094BDB6B236684F3098800F0BCFCAB
:103F000010B1064BA36110BD054BFBE783F311888D
:103F1000F9E700BF00ED00E000EF00E03F0300081C
:103F20004203000800F1604303F561430901C9B28F
:103F300083F80013012200F01F039A4043099B00FD
:103F400003F1604303F56143C3F880211A607047B1
:103F5000026843681143016003B1184770470000CD
:103F600013B5446BD4F894341A681178042915D128
:103F7000217C022912D11979128901238B40134225
:103F80000CD101A904F14C0001F09AFFD4F894443B
:103F9000019B21790246206800F0D0F902B010BDE3
:103FA000143001F01DBF00004FF0FF33143001F05A
:103FB00017BF00004C3001F0EFBF00004FF0FF339F
:103FC0004C3001F0E9BF0000143001F0EBBE0000FE
:103FD0004FF0FF31143001F0E5BE00004C3001F02D
:103FE000BBBF00004FF0FF324C3001F0B5BF000006
:103FF0000020704710B5D0F894341A68117804295D
:10400000044617D1017C022914D159795289012320
:104010008B4013420ED1143001F07EFE024648B1AF
:10402000D4F894444FF4807361792068BDE810405F
:1040300000F072B910BD0000406BFFF7DBBF00005D
:10404000704700007FB5124B036000234360C0E956
:104050000233012502260F4B05740446029001939A
:1040600000F18402294600964FF48073143001F069
:104070002FFE094B0294CDE9006304F523724FF43F
:104080008073294604F14C0001F0F6FE04B070BDC7
:10409000E467000839400008613F00080B683022DF
:1040A00082F311880A7903EB820290614A7909321E
:1040B00043F822008A7912B103EB8203986102234C
:1040C000C0F894140374002080F311887047000036
:1040D00038B5037F044613B190F85430ABB9201DB6
:1040E00001250221FFF734FF04F1140025776FF05A
:1040F000010100F079FC84F8545004F14C006FF099
:104100000101BDE8384000F06FBC38BD10B5012199
:1041100004460430FFF71CFF0023237784F8543053
:1041200010BD000038B504460025143001F0E8FD4C
:1041300004F14C00257701F0B7FE201D84F854509F
:104140000121FFF705FF2046BDE83840FFF752BFC9
:1041500090F8443003F06003202B07D190F84520FD
:10416000212A4FF0000303D81F2A06D800207047E9
:10417000222AFBD1C0E90E3303E0034A82630722FF
:10418000C2630364012070471D23002037B5D0F8B7
:1041900094341A681178042904461AD1017C022942
:1041A00017D11979128901238B40134211D100F1E3
:1041B0004C05284601F038FF58B101A9284601F006
:1041C0007FFED4F89444019B21790246206800F0D8
:1041D000B5F803B030BD0000F0B500EB810385B049
:1041E0009E6904460D46FEB1302383F3118804EB2B
:1041F0008507301D0821FFF7ABFEFB685B691B6874
:1042000006F14C001BB1019001F068FE019803A972
:1042100001F056FE024648B1039B2946204600F0B5
:104220008DF8002383F3118805B0F0BDFB685A694F
:104230001268002AF5D01B8A013B1340F1D104F12A
:104240004402EAE7093138B550F82140DCB13023A7
:1042500083F31188D4F894241368527903EB820312
:10426000DB689B695D6845B104216018FFF770FE4B
:10427000294604F1140001F059FD2046FFF7BAFE6B
:10428000002383F3118838BD7047000001F0CEB8D9
:10429000012303700023C0E90133C3618362036219
:1042A000C36243620363704738B50446302383F327
:1042B00011880025C0E90355C0E90555416001F0AA
:1042C000C5F80223237085F31188284638BD000005
:1042D00070B500EB810305465069DA600E4614465E
:1042E00018B110220021FDF7DDFAA06918B11022E3
:1042F0000021FDF7D7FA31462846BDE8704001F0AD
:104300006FB90000826802F0011282600022C0E9E9
:104310000422826101F0F0B9F0B400EB8104478916
:10432000E4680125A4698D403D4345812360002355
:10433000A2606360F0BC01F00BBA0000F0B400EBC7
:1043400081040789E468012564698D403D43058146
:1043500023600023A2606360F0BC01F085BA000016
:1043600070B50223002504460370C0E90255C0E978
:104370000455C564856180F8345001F0CDF8636858
:104380001B6823B129462046BDE87040184770BD20
:104390000378052B10B504460AD080F85030052369
:1043A000037043681B680BB1042198470023A36086
:1043B00010BD00000178052906D190F8502043680F
:1043C00002701B6803B118477047000070B590F881
:1043D0003430044613B1002380F8343004F1440231
:1043E000204601F0ABF963689B68B3B994F8443098
:1043F00013F0600535D00021204601F04BFC002170
:10440000204601F03DFC63681B6813B1062120467D
:104410009847062384F8343070BD2046984700281A
:10442000E4D0B4F84A30E26B9A4288BFE36394F96F
:104430004430E56B002B4FF0300380F20381002DF8
:1044400000F0F280092284F8342083F311880021DF
:10445000D4E90E232046FFF771FF002383F3118870
:10446000DAE794F8452003F07F0343EA022340F2A1
:104470000232934200F0C58021D8B3F5807F48D046
:104480000DD8012B3FD0022B00F09380002BB2D12E
:1044900004F14C02A2630222E2632364C1E7B3F594
:1044A000817F00F09B80B3F5407FA4D194F8463023
:1044B000012BA0D1B4F84C3043F0020332E0B3F545
:1044C000006F4DD017D8B3F5A06F31D0A3F5C063FE
:1044D000012B90D8636894F846205E6894F84710E2
:1044E000B4F848302046B047002884D04368A3631E
:1044F0000368E3631AE0B3F5106F36D040F602426A
:1045000093427FF478AF5C4BA3630223E363002301
:10451000C3E794F84630012B7FF46DAFB4F84C300C
:1045200023F00203C4E90E55A4F84C30256478E763
:10453000B4F84430B3F5A06F0ED194F8463084F847
:104540004E30204601F040F863681B6813B101212A
:1045500020469847032323700023C4E90E339CE7C9
:1045600004F14F03A3630123C3E72378042B10D185
:10457000302383F311882046FFF7C4FE85F31188AA
:104580000321636884F84F5021701B680BB12046EB
:10459000984794F84630002BDED084F84F3004233F
:1045A000237063681B68002BD6D0022120469847F1
:1045B000D2E794F848301D0603F00F0120460AD5D3
:1045C00001F0AEF8012804D002287FF414AF2B4B81
:1045D0009AE72B4B98E701F095F8F3E794F846300B
:1045E000002B7FF408AF94F8483013F00F01B3D0DC
:1045F0001A06204602D501F061FBADE701F054FB3D
:10460000AAE794F84630002B7FF4F5AE94F84830D2
:1046100013F00F01A0D01B06204602D501F03AFB93
:104620009AE701F02DFB97E7142284F8342083F3F6
:1046300011882B462A4629462046FFF76DFE85F352
:104640001188E9E65DB1152284F8342083F31188DE
:104650000021D4E90E232046FFF75EFEFDE60B2283
:1046600084F8342083F311882B462A4629462046B5
:10467000FFF764FEE3E700BF146800080C68000859
:104680001068000838B590F834300446002B3ED04E
:10469000063BDAB20F2A34D80F2B32D8DFE803F00A
:1046A000373131082232313131313131313137371F
:1046B000C56BB0F84A309D4214D2C3681B8AB5FB63
:1046C000F3F203FB12556DB9302383F311882B46A7
:1046D0002A462946FFF732FE85F311880A2384F81B
:1046E00034300EE0142384F83430302383F31188FF
:1046F00000231A4619462046FFF70EFE002383F3D7
:10470000118838BD036C03B198470023E7E7002107
:10471000204601F0BFFA0021204601F0B1FA63689B
:104720001B6813B10621204698470623D7E70000EF
:1047300010B590F83430142B044629D017D8062B26
:1047400005D001D81BB110BD093B022BFBD80021BD
:10475000204601F09FFA0021204601F091FA63689B
:104760001B6813B1062120469847062319E0152B34
:10477000E9D10B2380F83430302383F311880023F0
:104780001A461946FFF7DAFD002383F31188DAE7AA
:10479000C3689B695B68002BD5D1036C03B1984754
:1047A000002384F83430CEE7002303758268036960
:1047B0001B6899689142FBD25A680360426010609E
:1047C0005860704700230375826803691B68996805
:1047D0009142FBD85A68036042601060586070478D
:1047E00008B50846302383F311880B7D032B05D0D1
:1047F000042B0DD02BB983F3118808BD8B690022DF
:104800001A604FF0FF338361FFF7CEFF0023F2E71A
:10481000D1E9003213605A60F3E70000FFF7C4BF2C
:10482000054BD9680875186802681A605360012240
:104830000275D860FBF76EBD685C002030B50C4B8C
:10484000DD684B1C87B004460FD02B46094A6846EA
:1048500000F05EF92046FFF7E3FF009B13B16846C6
:1048600000F060F9A86907B030BDFFF7D9FFF9E79C
:10487000685C0020E1470008044B1A68DB68906818
:104880009B68984294BF002001207047685C00201C
:10489000084B10B51C68D86822681A605360012262
:1048A0002275DC60FFF78EFF01462046BDE8104010
:1048B000FBF730BD685C002038B5074C0749084855
:1048C000012300252370656001F0E6FB02232370BD
:1048D00085F3118838BD00BFD05E00201C68000839
:1048E000685C002008B572B6044B186500F048FCFF
:1048F00000F0FAFC024B03221A70FEE7685C00200D
:10490000D05E002000F044B9034A516853685B1A36
:104910009842FBD8704700BF001000E08B60022374
:1049200008618B82084670478368A3F1840243F8CC
:10493000142C026943F8442C426943F8402C094A7C
:1049400043F8242CC26843F8182C022203F80C2CDC
:10495000002203F80B2C044A43F8102CA3F120008A
:10496000704700BF2D030008685C002008B5FFF702
:10497000DBFFBDE80840FFF751BF0000024BDB68DA
:1049800098610F20FFF74CBF685C0020302383F351
:104990001188FFF7F3BF000008B50146302383F309
:1049A00011880820FFF74AFF002383F3118808BD10
:1049B000064BDB6839B1426818605A601360436087
:1049C0000420FFF73BBF4FF0FF307047685C0020CA
:1049D0000368984206D01A680260506099611846D0
:1049E000FFF71CBF7047000038B504460D4620682D
:1049F000844200D138BD036823605C608561FFF7A5
:104A00000DFFF4E710B503689C68A2420CD85C68FF
:104A10008A600B604C602160596099688A1A9A60BC
:104A20004FF0FF33836010BD1B68121BECE70000E2
:104A30000A2938BF0A2170B504460D460A266019B6
:104A400001F024FB01F010FB041BA54203D8751CE8
:104A50002E460446F3E70A2E04D9BDE87040012033
:104A600001F05ABB70BD0000F8B5144B0D46D9617A
:104A700003F1100141600A2A1969826038BF0A22D5
:104A8000016048601861A818144601F0F1FA0A277D
:104A900001F0EAFA431BA342064606D37C1C281900
:104AA00001F0F4FA27463546F2E70A2F04D9BDE8AB
:104AB000F840012001F030BBF8BD00BF685C002069
:104AC000F8B506460D4601F0CFFA0F4A134653F8E3
:104AD000107F9F4206D12A4601463046BDE8F84085
:104AE000FFF7C2BFD169BB68441A2C1928BF2C46F6
:104AF000A34202D92946FFF79BFF224631460348CD
:104B0000BDE8F840FFF77EBF685C0020785C0020BD
:104B100010B4C0E9032300235DF8044B4361FFF7A1
:104B2000CFBF000010B5194C236998420DD0D0E9D1
:104B30000032816813605A609A680A449A600023C0
:104B400003604FF0FF33A36110BD2346026843F8B2
:104B5000102F53600022026022699A4203D1BDE8FF
:104B6000104001F08DBA936881680B44936001F0A6
:104B70007BFA2269E1699268441AA242E4D911449D
:104B8000BDE81040091AFFF753BF00BF685C002062
:104B90002DE9F047DFF8BC8008F110072C4ED8F85B
:104BA000105001F061FAD8F81C40AA68031B9A4221
:104BB0003ED81444D5E900324FF00009C8F81C4033
:104BC00013605A60C5F80090D8F81030B34201D194
:104BD00001F056FA89F31188D5E903312846984740
:104BE000302383F311886B69002BD8D001F03CFA95
:104BF0006A69A0EB04094A4582460DD2022001F001
:104C00008BFA0022D8F81030B34208D1514628461A
:104C1000BDE8F047FFF728BF121A2244F2E712EB73
:104C2000090938BF4A4629463846FFF7EBFEB5E783
:104C3000D8F81030B34208D01444211AC8F81C0028
:104C4000A960BDE8F047FFF7F3BEBDE8F08700BFFD
:104C5000785C0020685C002038B501F005FA054A50
:104C6000D2E90845031B181945F10001C2E9080102
:104C700038BD00BF685C002000207047FEE70000E0
:104C8000704700004FF0FF307047000002290CD041
:104C9000032904D00129074818BF00207047032AC0
:104CA00005D8054800EBC200704704487047002053
:104CB000704700BFF46800082C230020A868000893
:104CC00070B59AB00546084601A9144600F0C2F82E
:104CD00001A8FCF7DFFD431C5B00C5E9003400229E
:104CE000237003236370C6B201AB02341046D1B205
:104CF0008E4204F1020401D81AB070BD13F8011BF2
:104D000004F8021C04F8010C0132F0E708B5302366
:104D100083F311880348FFF739FA002383F31188DE
:104D200008BD00BFD85E002090F8443003F01F0299
:104D3000012A07D190F845200B2A03D10023C0E9AE
:104D40000E3315E003F06003202B08D1B0F8483093
:104D50002BB990F84520212A03D81F2A04D8FFF741
:104D6000F7B9222AEBD0FAE7034A82630722C2632B
:104D700003640120704700BF2423002007B50529E4
:104D800017D8DFE801F0191603191920302383F32F
:104D90001188104A01900121FFF79AFA01980E4AF2
:104DA0000221FFF795FA0D48FFF7BCF9002383F3C2
:104DB000118803B05DF804FB302383F311880748A2
:104DC000FFF786F9F2E7302383F311880348FFF7F2
:104DD0009DF9EBE7486800086C680008D85E002081
:104DE00038B50C4D0C4C0D492A4604F10800FFF76C
:104DF00067FF05F1CA0204F110000949FFF760FFDF
:104E000005F5CA7204F118000649BDE83840FFF7FD
:104E100057BF00BFA06300202C2300202868000893
:104E2000326800083D68000870B5044608460D4623
:104E3000FCF730FDC6B22046013403780BB91846A2
:104E400070BD32462946FCF711FD0028F3D1012040
:104E5000F6E700002DE9F84F05460C46FCF71AFD71
:104E60002B49C6B22846FFF7DFFF08B10536F6B278
:104E700028492846FFF7D8FF08B11036F6B2632E4E
:104E80000DD8DFF88C80DFF88C90234FDFF890A0EE
:104E9000DFF890B02E7846B92670BDE8F88F294625
:104EA0002046BDE8F84F01F015BC252E2BD1072276
:104EB00041462846FCF7DAFC58B9DBF8003023609D
:104EC000DBF804306360DBF80830A36007350C348E
:104ED000E0E7082249462846FCF7C8FC98B90F4B82
:104EE000A21C197809090232C95D02F8041C13F8E2
:104EF000011B01F00F015345C95D02F8031CF0D1FD
:104F000018340835C6E704F8016B0135C2E700BF65
:104F1000146900083D68000829690008107AFF1F1D
:104F20001C7AFF1F1C690008BFF34F8F024AD36829
:104F3000DB03FCD4704700BF003C024008B5094BBE
:104F40001B7873B9FFF7F0FF074B1A69002ABFBF40
:104F5000064A5A6002F188325A601A6822F4806266
:104F60001A6008BDFE650020003C02402301674531
:104F700008B50B4B1B7893B9FFF7D6FF094B1A699D
:104F800042F000421A611A6842F480521A601A68AC
:104F900022F480521A601A6842F480621A6008BDD6
:104FA000FE650020003C02400728F0B516D80C4CE6
:104FB0000C4923787BB90C4D0E4608234FF0006254
:104FC00055F8047B46F8042B013B13F0FF033A44E9
:104FD000F6D10123237051F82000F0BD0020FCE73A
:104FE00020660020006600203C690008014B53F851
:104FF000200070473C69000808207047072810B55A
:10500000044601D9002010BDFFF7CEFF064B53F830
:1050100024301844C21A0BB90120F4E71268013297
:10502000F0D1043BF6E700BF3C690008072810B543
:10503000044621D8FFF778FFFFF780FF0F4AF323DC
:10504000D360C300DBB243F4007343F00203136187
:10505000136943F480331361FFF766FFFFF7A4FF82
:10506000074B53F8241000F03BF9FFF781FF20466F
:10507000BDE81040FFF7C2BF002010BD003C024059
:105080003C690008F8B512F00103144642D18518B6
:105090002E4A954257D82E4B1B6813F0010352D06D
:1050A0002C4DFFF74BFFF323EB60FFF73DFF40F282
:1050B0000127032C15D824F001046618254C401A4A
:1050C00040F20117B142236900EB010524D123F01E
:1050D00001032361FFF74CFF0120F8BD043C0430BD
:1050E000E7E78307E7D12B6923F440732B612B6932
:1050F0003B432B6151F8046B0660BFF34F8FFFF702
:1051000013FF03689E42E9D02B6923F001032B6152
:10511000FFF72EFF0020E0E723F4407323612369AB
:105120003B4323610B882B80BFF34F8FFFF7FCFEBF
:105130002D8831F8023BADB2AB42C3D0236923F0D6
:1051400001032361E4E71846C7E700BF0000080831
:1051500000380240003C0240084908B50B7828B1ED
:105160001BB9FFF7EBFE01230B7008BD002BFCD031
:10517000BDE808400870FFF7FBBE00BFFE650020D9
:1051800008B50649064800F0ADF8BDE808404FF400
:1051900080314FF0805000F0A5B800BF00FF010043
:1051A000000100200846114601F044BA084601F00B
:1051B00057BA000038B5EFF311859DB9EFF30584B8
:1051C000C4F30804302334B183F31188FFF744FD9E
:1051D00085F3118838BD83F31188FFF73DFD84F313
:1051E000118838BDBDE83840FFF736BD38B5FFF748
:1051F000E1FF114C114AC00840EA4170A0FB025E79
:10520000C908A0FB040C1CEB050CA1FB04404FF0EB
:1052100000035B41A1FB02121CEB040C43EB0000FA
:1052200011EB0E0142F10002411842F100000909A0
:1052300041EA007038BD00BFCFF753E3A59BC420FF
:1052400010B50244064BD2B2904200D110BD441CAE
:1052500000B253F8200041F8040BE0B2F4E700BFBD
:10526000502800400F4B30B51C6F240407D41C6F2E
:1052700044F400741C671C6F44F400441C670A4C1F
:10528000236843F4807323600244084BD2B29042F7
:1052900000D130BD441C00B251F8045B43F82050EB
:1052A000E0B2F4E7003802400070004050280040AF
:1052B00007B5012201A90020FFF7C2FF019803B042
:1052C0005DF804FB13B50446FFF7F2FFA04205D0DA
:1052D000012201A900200194FFF7C4FF02B010BD14
:1052E000704700007047000070470000074B45F210
:1052F00055521A6003225A6040F2FF729A604CF6CF
:10530000CC421A60024B01221A70704700300040F4
:1053100028660020034B1B781BB1034B4AF6AA22D8
:105320001A6070472866002000300040034B1A685E
:105330001AB9034AD2F874281A607047246600200C
:1053400000300240024B4FF08072C3F8742870475F
:105350000030024008B5FFF7E9FF024B1868C0F3C0
:10536000407008BD2466002008B5FFF7DFFF024B40
:105370001868C0F3007008BD246600207047000064
:10538000FEE700000A4B0B480B4A90420BD30B4B35
:10539000DA1C121AC11E22F003028B4238BF00220F
:1053A0000021FCF77FBA53F8041B40F8041BECE71C
:1053B000486B000824670020246700202467002031
:1053C00070B5D0E915439E6800224FF0FF3504EB1D
:1053D00042135101D3F800090028BEBFD3F80009D9
:1053E00040F08040C3F80009D3F8000B0028BEBF8E
:1053F000D3F8000B40F08040C3F8000B0132631873
:105400009642C3F80859C3F8085BE0D24FF0011385
:10541000C4F81C3870BD0000890141F02001016111
:1054200003699B06FCD41220FFF76EBA10B5054C39
:105430002046FEF72DFF4FF0A0436365024BA365A6
:1054400010BD00BF2C6600208069000870B503788D
:10545000012B054650D12A4B446D98421BD1294B54
:105460005A6B42F080025A635A6D42F080025A65CC
:105470005A6D5A6942F080025A615A6922F08002DC
:105480005A610E2143205B69FEF74CFD1E4BE36021
:105490001E4BC4F800380023C4F8003EC02323602C
:1054A0006E6D4FF40413A3633369002BFCDA012300
:1054B00033610C20FFF728FA3369DB07FCD4122094
:1054C000FFF722FA3369002BFCDA0026A660284693
:1054D000FFF776FF6B68C4F81068DB68C4F81468DF
:1054E000C4F81C684BB90A4BA3614FF0FF336361EA
:1054F000A36843F00103A36070BD064BF4E700BF4F
:105500002C660020003802404014004003002002B6
:10551000003C30C0083C30C0F8B5446D0546002161
:105520002046FFF779FFA96D00234FF001128F6825
:10553000C4F834384FF00066C4F81C284FF0FF3030
:1055400004EB431201339F42C2F80069C2F8006BBA
:10555000C2F80809C2F8080BF2D20B686A6DEB6555
:10556000636210231361166916F01006FBD1122036
:10557000FFF7CAF9D4F8003823F4FE63C4F8003802
:10558000A36943F4402343F01003A3610923C4F843
:105590001038C4F814380A4BEB604FF0C043C4F81D
:1055A000103B084BC4F8003BC4F81069C4F800393C
:1055B000EB6D03F1100243F48013EA65A362F8BDBA
:1055C0005C69000840800010426D90F84E10D2F8DF
:1055D000003823F4FE6343EA0113C2F80038704731
:1055E0002DE9F84300EB8103456DDA68166806F093
:1055F0000306731E022B05EB41130C4680460FFA7F
:1056000081F94FEA41104FF00001C3F8101B4FF031
:10561000010104F1100398BFB60401FA03F3916984
:105620008EBF334E06F1805606F5004600293AD06B
:10563000578A04F15801490137436F50D5F81C18B7
:105640000B43C5F81C382B180021C3F810195369F7
:105650000127611EA7409BB3138A928B9B08012AE6
:1056600088BF5343D8F85C20981842EA034301F1FD
:10567000400205EB8202C8F85C00214653602846D0
:10568000FFF7CAFE08EB8900C3681B8A43EA84530C
:10569000483464011E432E51D5F81C381F43C5F809
:1056A0001C78BDE8F88305EB4917D7F8001B21F4F7
:1056B0000041C7F8001BD5F81C1821EA0303C0E716
:1056C00004F13F0305EB83030A4A5A60284621464A
:1056D000FFF7A2FE05EB4910D0F8003923F4004390
:1056E000C0F80039D5F81C3823EA0707D7E700BF10
:1056F0000080001000040002826D1268C265FFF78E
:105700005FBE00005831436D49015B5813F40040FF
:1057100004D013F4001F0CBF0220012070470000CA
:105720004831436D49015B5813F4004004D013F431
:10573000001F0CBF022001207047000000EB810118
:10574000CB68196A0B6813604B68536070470000A0
:1057500000EB810330B5DD68AA691368D36019B91D
:10576000402B84BF402313606B8A1468426D1C4435
:10577000013CB4FBF3F46343033323F0030302EB74
:10578000411043EAC44343F0C043C0F8103B2B68C8
:1057900003F00303012B09B20ED1D2F8083802EB53
:1057A000411013F4807FD0F8003B14BF43F08053C6
:1057B00043F00053C0F8003B02EB4112D2F8003B2B
:1057C00043F00443C2F8003B30BD00002DE9F04136
:1057D000244D6E6D06EB40130446D3F8087BC3F8E6
:1057E000087B38070AD5D6F81438190706D505EB13
:1057F00084032146DB6828465B689847FA071FD573
:10580000D6F81438DB071BD505EB8403D968CCB96F
:105810008B69488A5A68B2FBF0F600FB16228AB9F7
:105820001868DA6890420DD2121AC3E900243023B6
:1058300083F311880B482146FFF78AFF84F3118810
:10584000BDE8F081012303FA04F26B8923EA020325
:105850006B81CB68002BF3D021460248BDE8F041B4
:10586000184700BF2C66002000EB810370B5DD688F
:10587000436D6C692668E6604A0156BB1A444FF4D2
:105880000020C2F810092A6802F00302012A0AB2B5
:105890000ED1D3F8080803EB421410F4807FD4F83B
:1058A000000914BF40F0805040F00050C4F80009D7
:1058B00003EB4212D2F8000940F00440C2F800099C
:1058C000D3F83408012202FA01F10143C3F8341875
:1058D00070BD19B9402E84BF4020206020682E8AF8
:1058E0008419013CB4FBF6F440EAC44040F0005097
:1058F0001A44C6E72DE9F8433B4D6E6D06EB4013A5
:105900000446D3F80889C3F8088918F0010F4FEA54
:1059100040171AD0D6F81038DB0716D505EB8003F0
:10592000D9684B691868DA68904230D2121A4FF081
:1059300000091A60C3F80490302383F311882146CC
:105940002846FFF791FF89F3118818F0800F1CD0CB
:10595000D6F834380126A640334216D005EB84032E
:105960006D6DD3F80CC0DCF814200134E4B2D2F829
:1059700000E005EB04342F445168714515D3D5F888
:10598000343823EA0606C5F83468BDE8F8830123F5
:1059900003FA04F22B8923EA02032B818B68002B84
:1059A000D3D0214628469847CFE7BCF81000AEEB8D
:1059B0000103834228BF0346D7F8180980B2B3EB2E
:1059C000800FE2D89068A0F1040959F8048FC4F858
:1059D0000080A0EB09089844B8F1040FF5D81844EA
:1059E0000B4490605360C7E72C6600202DE9F74F09
:1059F000A24C656D6E69AB691E4016F480586E61ED
:105A000007D02046FEF7ACFC03B0BDE8F04FFEF730
:105A10005FBA002E12DAD5F8003E98489B071EBFE9
:105A2000D5F8003E23F00303C5F8003ED5F804384E
:105A300023F00103C5F80438FEF7BCFC370505D593
:105A40008E48FFF7BDFC8D48FEF7A2FCB0040CD5D4
:105A5000D5F8083813F0060FEB6823F470530CBF29
:105A600043F4105343F4A053EB6031071BD5636834
:105A7000DB681BB9AB6923F00803AB612378052B06
:105A80000CD1D5F8003E7D489A071EBFD5F8003EE0
:105A900023F00303C5F8003EFEF78CFC6368DB6867
:105AA0000BB176489847F30274D4B70227D5D4F8DF
:105AB0005490DFF8C8B100274FF0010A09EB4712F4
:105AC000D2F8003B03F44023B3F5802F11D1D2F874
:105AD000003B002B0DDA62890AFA07F322EA03037E
:105AE000638104EB8703DB68DB6813B139465846F2
:105AF0009847A36D01379B68FFB29F42DED9F0063D
:105B000017D5676D3A6AC2F30A1002F00F0302F468
:105B1000F012B2F5802F00F08580B2F5402F08D149
:105B200004EB83030022DB681B6A07F58057904271
:105B30006AD13003D5F8184813D5E10302D5002007
:105B4000FFF744FEA20302D50120FFF73FFE6303E7
:105B500002D50220FFF73AFE270302D50320FFF704
:105B600035FE75037FF550AFE00702D50020FFF743
:105B7000C1FEA10702D50120FFF7BCFE620702D5D6
:105B80000220FFF7B7FE23077FF53EAF0320FFF7A4
:105B9000B1FE39E7636DDFF8E4A0019300274FF011
:105BA0000109A36D9B685FFA87FB9B453FF67DAFBC
:105BB000019B03EB4B13D3F8001901F44021B1F51D
:105BC000802F1FD1D3F8001900291BDAD3F8001950
:105BD00041F09041C3F80019D3F800190029FBDB0C
:105BE0005946606DFFF718FC218909FA0BF321EA89
:105BF0000303238104EB8B03DB689B6813B15946D5
:105C0000504698470137CCE7910708BFD7F8008086
:105C1000072A98BF03F8018B02F1010298BF4FEAEF
:105C2000182884E7023304EB830207F58057526893
:105C3000D2F818C0DCF80820DCE9001CA1EB0C0C41
:105C4000002188420AD104EB830463689B699A6847
:105C500002449A605A6802445A606AE711F0030FDE
:105C600008BFD7F800808C4588BF02F8018B01F18E
:105C7000010188BF4FEA1828E3E700BF2C66002027
:105C8000436D03EB4111D1F8003B43F40013C1F81D
:105C9000003B7047436D03EB4111D1F8003943F4E9
:105CA0000013C1F800397047436D03EB4111D1F87F
:105CB000003B23F40013C1F8003B7047436D03EB36
:105CC0004111D1F8003923F40013C1F800397047AD
:105CD00030B5039C0172043304FB0325C0E906536D
:105CE000049B03630021059BC160C0E90000C0E97B
:105CF0000422C0E90842C0E90A11436330BD000034
:105D0000416A0022C0E90411C0E90A22C2606FF0B2
:105D10000101FEF769BE0000D0E90432934201D1CF
:105D2000C2680AB9181D70470020704703691960DE
:105D3000C2680132C260C26913448269036193423E
:105D400024BF436A03610021FEF742BE38B5044612
:105D50000D46E3683BB16269131D1268A3621344E8
:105D6000E362002007E0237A33B929462046FEF794
:105D70001FFE0028EDDA38BD6FF00100FBE70000E0
:105D8000C368C269013BC3604369134482694361CC
:105D9000934224BF436A436100238362036B03B1D0
:105DA0001847704770B53023044683F31188866A1C
:105DB0003EB9FFF7CBFF054618B186F31188284698
:105DC00070BDA36AE26A13F8015BA362934202D337
:105DD0002046FFF7D5FF002383F31188EFE700008B
:105DE0002DE9F84F04460E46174698464FF0300905
:105DF00089F311880025AA46D4F828B0BBF1000F1A
:105E000009D141462046FFF7A1FF20B18BF311884D
:105E10002846BDE8F88FD4E90A12A7EB050B521A01
:105E2000934528BF9346BBF1400F1BD9334601F180
:105E3000400251F8040B43F8040B9142F9D1A36AD4
:105E400040334036A3624035D4E90A239A4202D354
:105E50002046FFF795FF8AF31188BD42D8D289F317
:105E60001188C9E730465A46FBF7F6FCA36A5B4443
:105E70005E44A3625D44E7E710B5029C01720433FF
:105E800003FB0421C0E906130023C0E90A33039B86
:105E90000363049BC460C0E90000C0E90422C0E9B8
:105EA0000842436310BD0000026AC260426AC0E952
:105EB00004220022C0E90A226FF00101FEF794BD1E
:105EC000D0E904239A4201D1C26822B9184650F899
:105ED000043B0B60704700231846FAE7C368C269A9
:105EE0000133C3604369134482694361934224BF11
:105EF000436A43610021FEF76BBD000038B50446DC
:105F00000D46E3683BB123691A1DA262E26913449E
:105F1000E362002007E0237A33B929462046FEF7E2
:105F200047FD0028EDDA38BD6FF00100FBE7000007
:105F300003691960C268013AC260C2691344826988
:105F40000361934224BF436A036100238362036BAE
:105F500003B118477047000070B530230D46044662
:105F6000114683F31188866A2EB9FFF7C7FF10B177
:105F700086F3118870BDA36A1D70A36AE26A0133BB
:105F80009342A36204D3E16920460439FFF7D0FFAE
:105F9000002080F31188EDE72DE9F84F04460D4607
:105FA000904699464FF0300A8AF311880026B3468E
:105FB000A76A4FB949462046FFF7A0FF20B187F3F3
:105FC00011883046BDE8F88FD4E90A073A1AA8EBE1
:105FD0000607974228BF1746402F1BD905F14003FB
:105FE00055F8042B40F8042B9D42F9D1A36A4033A5
:105FF000A3624036D4E90A239A4204D3E1692046D9
:106000000439FFF795FF8BF311884645D9D28AF3FF
:106010001188CDE729463A46FBF71EFCA36A3B44AC
:106020003D44A3623E44E5E7D0E904239A4217D1F8
:10603000C3689BB1836A8BB1043B9B1A0ED013607B
:10604000C368013BC360C3691A44836902619A4211
:1060500024BF436A0361002383620123184670470B
:106060000023FBE700F0D2B84FF08043586A704736
:106070004FF08043002258631A610222DA607047B1
:106080004FF080430022DA60704700004FF08043F9
:1060900058637047FEE7000070B51B4B0163002595
:1060A000044686B0586085620E46FDF7EDFE04F1A9
:1060B0001003C4E904334FF0FF33C4E90635C4E9E3
:1060C0000044A560E562FFF7CFFF2B460246C4E916
:1060D000082304F134010D4A256580232046FEF78C
:1060E0001DFC0123E0600A4A037500927268019268
:1060F000B268CDE90223074B6846CDE90435FEF7C7
:1061000035FC06B070BD00BFD05E00208C69000871
:106110009169000895600008024AD36A1843D0626A
:10612000704700BF685C00204B6843608B688360E9
:10613000CB68C3600B6943614B6903628B6943623F
:106140000B6803607047000008B5264B26481A69A3
:1061500040F2FF110A431A611A6922F4FF7222F019
:1061600001021A611A691A6B0A431A631A6D0A430B
:106170001A651E4A1B6D1146FFF7D6FF02F11C017E
:1061800000F58060FFF7D0FF02F1380100F5806074
:10619000FFF7CAFF02F1540100F58060FFF7C4FF6A
:1061A00002F1700100F58060FFF7BEFF02F18C0183
:1061B00000F58060FFF7B8FF02F1A80100F58060EC
:1061C000FFF7B2FF02F1C40100F58060FFF7ACFFFA
:1061D00002F1E00100F58060FFF7A6FFBDE808408E
:1061E00000F090B8003802400000024098690008B2
:1061F00008B500F0FBF9FEF75FFBFFF797F8BDE885
:106200000840FEF7EDBD0000704700000F4B1A6C10
:1062100042F001021A641A6E42F001021A660C4A38
:106220001B6E936843F0010393604FF08043532249
:106230009A624FF0FF32DA6200229A615A63DA60A2
:106240005A6001225A611A60704700BF003802404C
:10625000002004E04FF0804208B51169D3680B407C
:10626000D9B2C9439B07116107D5302383F3118845
:10627000FEF748FB002383F3118808BD1F4B1A6902
:106280006FEAC2526FEAD2521A611A69C2F3080267
:106290001A614FF0FF301A695A69586100215A6932
:1062A00059615A691A6A62F080521A621A6A02F0D7
:1062B00080521A621A6A5A6A58625A6A59625A6A4B
:1062C0001A6C42F080521A641A6E42F080521A66BA
:1062D0001A6E0B4A106840F480701060186F00F45A
:1062E0004070B0F5007F1EBF4FF48030186719670B
:1062F000536823F40073536000F054B9003802402F
:1063000000700040334B4FF080521A64324A4FF411
:10631000404111601A6842F001021A601A68910740
:10632000FCD59A6822F003029A602A4B9A6812F010
:106330000C02FBD1196801F0F90119609A601A6822
:1063400042F480321A601A689203FCD55A6F42F008
:1063500001025A671F4B5A6F9007FCD51F4A5A60BB
:106360001A6842F080721A601B4A53685904FCD5BF
:10637000184B1A689201FCD5194A9A60194B1A6891
:10638000194B9A42194B21D1194A1168194A914265
:106390001CD140F205121A60144A136803F00F036F
:1063A000052BFAD10B4B9A6842F002029A609A6868
:1063B00002F00C02082AFAD15A6C42F480425A6464
:1063C0005A6E42F480425A665B6E704740F2057224
:1063D000E1E700BF00380240007000400854400769
:1063E00000948838002004E011640020003C024042
:1063F00000ED00E041C20F41074A08B5536903F0C0
:106400000103536123B1054A13680BB150689847E3
:10641000BDE80840FDF75CBD003C0140A4660020DB
:10642000074A08B5536903F00203536123B1054AD3
:1064300093680BB1D0689847BDE80840FDF748BDA8
:10644000003C0140A4660020074A08B5536903F0E8
:106450000403536123B1054A13690BB1506998478E
:10646000BDE80840FDF734BD003C0140A4660020B3
:10647000074A08B5536903F00803536123B1054A7D
:1064800093690BB1D0699847BDE80840FDF720BD7E
:10649000003C0140A4660020074A08B5536903F098
:1064A0001003536123B1054A136A0BB1506A984730
:1064B000BDE80840FDF70CBD003C0140A46600208B
:1064C000164B10B55C6904F478725A61A30604D5C2
:1064D000134A936A0BB1D06A9847600604D5104AF4
:1064E000136B0BB1506B9847210604D50C4A936B84
:1064F0000BB1D06B9847E20504D5094A136C0BB178
:10650000506C9847A30504D5054A936C0BB1D06C29
:106510009847BDE81040FDF7DBBC00BF003C0140E0
:10652000A4660020194B10B55C6904F47C425A61E2
:10653000620504D5164A136D0BB1506D98472305BB
:1065400004D5134A936D0BB1D06D9847E00404D580
:106550000F4A136E0BB1506E9847A10404D50C4A34
:10656000936E0BB1D06E9847620404D5084A136F3E
:106570000BB1506F9847230404D5054A936F0BB1B4
:10658000D06F9847BDE81040FDF7A2BC003C014029
:10659000A466002008B5FFF75DFEBDE80840FDF7E2
:1065A00097BC0000062108B50846FDF7BBFC062194
:1065B0000720FDF7B7FC06210820FDF7B3FC0621F4
:1065C0000920FDF7AFFC06210A20FDF7ABFC0621F0
:1065D0001720FDF7A7FC06212820FDF7A3FCBDE846
:1065E000084007211C20FDF79DBC000008B5FFF7FF
:1065F00045FE00F00BF8FDF749FEFDF721FDFFF722
:1066000003FEBDE80840FFF72DBD00000023054A4A
:1066100019460133102BC2E9001102F10802F8D12A
:10662000704700BFA46600200B460146184600F0E4
:1066300009B80000024B0A4601461868FEF7B2BDD1
:106640004C23002010B5054C13462CB10A460146D8
:106650000220AFF3008010BD2046FCE700000000E0
:10666000024B01461868FEF7A1BD00BF4C23002075
:1066700010B501390244904201D1002005E00378B1
:1066800011F8014FA34201D0181B10BD0130F2E7F1
:106690002DE9F041A3B1C91A17780144044603F16A
:1066A000FF3C8C42204601D9002009E00578BD421C
:1066B00004F10104F5D10CEB0405D618A54201D173
:1066C000BDE8F08115F8018D16F801EDF045F5D023
:1066D000E7E70000034611F8012B03F8012B002A1D
:1066E000F9D1704773772D737061722D663430372E
:1066F0002D626C0053544D3332463F3F3F0053549C
:106700004D3332463430780053544D3332463432B0
:10671000780053544D333246343436585800000014
:10672000012033000010410001105A0003105900ED
:106730000710310000000000F46600081304000098
:10674000FE66000819040000086700082104000024
:106750001267000840A2E4F1646891060041A3E5D5
:10676000F2656992070000004261642043414E498E
:106770006661636520696E6465782E000001000023
:106780000001FF000064004000680040800000003D
:1067900000800000000080000000000000000000F9
:1067A000F1210008DD2A0008E5290008312200084F
:1067B0003D22000849240008012200081122000897
:1067C000052200080D2200080922000865230008A0
:1067D00015220008352E0008E52D000825220008A6
:1067E0003923000800000000BD3F0008A93F000851
:1067F000E53F0008D13F0008DD3F0008C93F000821
:10680000B53F0008A13F0008F13F0008000000006C
:10681000010000000000000063300000186800085C
:10682000C05C0020D05E00204172647550696C6FBE
:10683000740025424F415244252D424C00255345BA
:106840005249414C250000000200000000000000F9
:10685000D941000845420008400040007063002014
:106860008063002002000000000000000300000020
:106870000000000089420008000000001000000035
:1068800090630020000000000100000000000000F4
:106890002C660020010102007D4D00088D4C00088F
:1068A000294D00080D4D000843000000B0680008A5
:1068B00009024300020100C0320904000001020283
:1068C0000100052400100105240100010424020236
:1068D0000524060001070582030800FF09040100E2
:1068E000020A0000000705010240000007058102BE
:1068F0004000000012000000FC68000812011001B6
:106900000200004009124157000201020301000089
:106910000403090425424F415244250073772D7327
:106920007061722D66343037003031323334353691
:1069300037383941424344454600000000400000DA
:106940000040000000400000004000000000010086
:106950000000020000000200000002000000000031
:10696000CD4300088546000831470008400040003C
:106970008C6600208C660020010000009C660020D0
:106980008000000040010000030000006D61696E9E
:106990000069646C650000000000802A00000000AF
:1069A000AAAAAAAA00000024FFFF0000000000001D
:1069B00000A00A000068000000000000AA6AAAAA5D
:1069C000000000007FFF00000000900900000000B0
:1069D0000000010000000000AAAAAAAA000000000E
:1069E000FFFE000000000000000000001A00000090
:1069F000000000009AAAAAAA00000000FFFF000001
:106A000099000000000000000000000000000000ED
:106A1000AAAAAAAA00000000FFFF000000000000D0
:106A2000000000000000000000000000AAAAAAAABE
:106A300000000000FFFF0000000000000000000058
:106A40000000000000000000AAAAAAAA000000009E
:106A5000FFFF000000000000000000000000000038
:106A6000000000000A000000000000000300000019
:106A70000000000000000000000000000000000016
:106A80000000000000000000000000000000000006
:106A9000000000000000000070170000000000006F
:106AA000000007000000000040420F00FE2A010025
:106AB000D2040000FF0096000000000800960000CD
:106AC0000000080004000000106900080000000039
:106AD00000000000000000000000000000000000B6
:106AE0000000000050230020000000000000000013
:106AF0000000000000000000000000000000000096
:106B00000000000000000000000000000000000085
:106B10000000000000000000000000000000000075
:106B20000000000000000000000000000000000065
:106B30000000000000000000000000000000000055
:086B400000000000000000004D
:00000001FF
